:0200000480007A
:10000000B72F0000938F0F8073900F306F00400365
:100010001300000013000000130000001300000094
:100020001300000013000000130000001300000084
:100030001300000013000000130000001300000074
:100040009702000093824211739052309300000097
:10005000130100009301000013020000930200004E
:100060001303000093030000130400009304000036
:10007000130500009305000013060000930600001E
:100080001307000093070000130800009308000006
:100090001309000093090000130A0000930A0000EE
:1000A000130B0000930B0000130C0000930C0000D6
:1000B000130D0000930D0000130E0000930E0000BE
:1000C000130F0000930F000097110200938141C4A9
:1000D0001705020013050547979503009385456EA4
:1000E00013060000EF00001A170502001305C538BB
:1000F000970502009385854113060000EF008018E4
:1001000017A503001305056C97B503009385456B90
:1001100037B6ABAB1306B6BAEF00C01617B1030083
:100120001301416AEF80101E9392120093D21200C5
:100130009382D2FF638A02008322010013014100EF
:100140006F0000177300203083220100130141006B
:10015000730020301301C1FF23205100F32220340B
:10016000E3C402FC8322010013014100130141F8A2
:1001700023221100232421002326310023284100BB
:10018000232A5100232C6100232E71002320810299
:10019000232291022324A1022326B1022328C10293
:1001A000232AD102232CE102232EF1022320010570
:1001B0002322110523242105232631052328410567
:1001C000232A5105232C6105232E71052320810745
:1001D000232291072324A1072326B1072328C1073F
:1001E000232AD107232CE107232EF107732520347E
:1001F000F3251034130601006F000000731015344E
:1002000083204100032181008321C10003220101D9
:1002100083224101032381018323C10103240102BD
:1002200083244102032581028325C10203260103A1
:1002300083264103032781038327C1030328010485
:1002400083284104032981048329C104032A010569
:10025000832A4105032B8105832BC105032C01064D
:10026000832C4106032D8106832DC106032E010731
:10027000832E4107032F8107832FC1071301C10775
:10028000730020302320C5006376B50013054500B8
:100290006FF05FFF678000000000000000000000BA
:1002A000000000000000000000000000000000004E
:1002B000130101F8232011002322210023243100FF
:1002C0002326410023285100232A6100232C71009A
:1002D000232E8100232091022322A1022324B10294
:1002E0002326C1022328D102232AE102232CF10272
:1002F000232E010323201105232221052324310568
:100300002326410523285105232A6105232C710545
:10031000232E8105232091072322A1072324B1073F
:100320002326C1072328D107232AE107232CF1071D
:100330009702020083A2821723A02200F322103426
:10034000232E5106EF00C03B1701020003210116C6
:10035000032101008322C10773901234B7220000E9
:100360009382028873A00230832001000322C1001F
:100370008322010103234101832381010324C1015D
:100380008324010203254102832581020326C10241
:100390008326010303274103832781030328C10325
:1003A000832801040329410483298104032AC10409
:1003B000832A0105032B4105832B8105032CC105ED
:1003C000832C0106032D4106832D8106032EC106D1
:1003D000832E0107032F4107832F81071301010893
:1003E00073002030970202009382C21523A01200EE
:1003F00023A2220023A4320023A6420023A85200F5
:1004000023AA620023AC720023AE820023A09202D2
:1004100023A2A20223A4B20223A6C20223A8D202CC
:1004200023AAE20223ACF20223AE020323A01205A8
:1004300023A2220523A4320523A6420523A85205A0
:1004400023AA620523AC720523AE820523A092077E
:1004500023A2A20723A4B20723A6C20723A8D20778
:1004600023AAE20723ACF207EF601036170102005F
:100470000321C103032101008322C10773901234B9
:10048000B72200009382028873A00230832001000B
:100490000322C1008322010103234101832381013F
:1004A0000324C10183240102032541028325810223
:1004B0000326C10283260103032741038327810307
:1004C0000328C103832801040329410483298104EB
:1004D000032AC104832A0105032B4105832B8105CF
:1004E000032CC105832C0106032D4106832D8106B3
:1004F000032EC106832E0107032F4107832F810797
:1005000013010108730020309702020093828203D6
:1005100083A0020003A1420083A1820003A2C200C3
:1005200083A2020103A3420183A3820103A4C201A7
:1005300083A4020203A5420283A5820203A6C2028B
:1005400083A6020303A7420383A7820303A8C2036F
:1005500083A8020403A9420483A9820403AAC20453
:1005600083AA020503AB420583AB820503ACC20537
:1005700083AC020603AD420683AD820603AEC2061B
:1005800083AE020703AFC20983AF82076780000012
:1005900073700430130101F823201100232221007D
:1005A000232431002326410023285100232A6100FF
:1005B000232C7100232E8100232091022322A102EB
:1005C0002324B1022326C1022328D102232AE102D7
:1005D000232CF102232E01032320110523222105C0
:1005E000232431052326410523285105232A6105AB
:1005F000232C7105232E8105232091072322A10797
:100600002324B1072326C1072328D107232AE10782
:10061000232CF1079702020083A242E923A02200C3
:10062000232E1106EF30402817010200032101E8B4
:10063000032101008322C10773901234B722000006
:100640009382028873A00230832001000322C1003C
:100650008322010103234101832381010324C1017A
:100660008324010203254102832581020326C1025E
:100670008326010303274103832781030328C10342
:10068000832801040329410483298104032AC10426
:10069000832A0105032B4105832B8105032CC1050A
:1006A000832C0106032D4106832D8106032EC106EE
:1006B000832E0107032F4107832F810713010108B0
:1006C00073002030737004306F00000073104530E9
:1006D000678000007325403073F04330678000006E
:1006E00097070000938747FE232EB5FE2322C5FA05
:1006F000232635F82320F5F8130505F86780000058
:10070000130101FF23261100EF60D008EF20805075
:10071000631805008320C1001301010167800000F8
:100720008320C100130101016F3000189307850079
:100730001307F0FF2322F5002324E5002326F5000C
:100740002328F500232005006780000023280500EA
:10075000678000008327450023A2F50003A78700D8
:1007600023A4E50003A787002322B70023A4B70032
:1007700023A8A50083270500938717002320F500F1
:100780006780000003A605009307F0FF13078500AC
:100790006316F6006F008003138707008327470066
:1007A00083A60700E37AD6FE23A2F50023A4B700B0
:1007B00023A4E5002322B70023A8A5008327050072
:1007C000938717002320F5006780000003270501A9
:1007D000832747006FF05FFD0327450083268500D0
:1007E000832705012324D70003278500832645009E
:1007F0002322D70003A747006316A700032785001D
:1008000023A2E7002328050003A507001305F5FF31
:1008100023A0A70067800000032605049387050036
:10082000630406028325C50003274500B385C50080
:100830002326B50063E6E500832505002326B500E1
:10084000138507006F50405167800000130101FFBE
:100850002324810023261100130405002322910084
:10086000EF30D03783278404635AF004832744028F
:1008700063860704930444026F0000028327840404
:100880009387F7FF2324F404832784046358F0023A
:10089000832744026384070213850400EF3000635A
:1008A000E30E05FCEF30D00F832784049387F7FF16
:1008B0002324F40483278404E34CF0FC9307F0FF23
:1008C0002324F404EF30D034EF3050318327440434
:1008D000635AF00483270401638607049304040128
:1008E0006F000002832744049387F7FF2322F40458
:1008F000832744046358F0028327040163840702BA
:1009000013850400EF30805CE30E05FCEF305009E6
:10091000832744049387F7FF2322F40483274404A6
:10092000E34CF0FC9307F0FF2322F404032481003E
:100930008320C10083244100130101016F30502D39
:1009400063000508130101FF232481002322910085
:10095000130405002326110093840500EF301028AE
:10096000832604048327C40303270400232C0402E2
:10097000B387F6021306F0FF2322C4042324E40005
:100980002324C404B386D740B307F7003307D70046
:100990002322F4002326E400639804028327040141
:1009A000639E0702EF30D0268320C100032481001C
:1009B000832441001305100013010101678000002A
:1009C000737004306F00000013050401EFF01FD6B0
:1009D00013054402EFF09FD56FF0DFFC130504010F
:1009E000EF30C04E93071000E31EF5FAEFF05FBA48
:1009F0006FF05FFB63160500737004306F0000003A
:100A0000130101FE232A910023282101232631010D
:100A1000232E1100232C8100930906001389050061
:100A200093040500638E05083305B50213055505CB
:100A3000EF50001213040500630C050893074505E9
:100A40002320F500232E940223202405EF301019D3
:100A5000832604048327C403032704001306F0FF3E
:100A6000B387F602232C04022322C4042324E400C7
:100A70002324C40413050401B386D740B307F70049
:100A80003307D7002322F4002326E400EFF01FCA27
:100A900013054402EFF09FC9EF3090172308340587
:100AA000130504008320C101032481018324410133
:100AB000032901018329C10013010102678000009D
:100AC00013054005EF50C008130405006316050028
:100AD000737004306F000000232084006FF09FF6D5
:100AE00063160500737004306F0000006376B50074
:100AF000737004306F000000130101FF2324810094
:100B0000130620001384050093050000232611001E
:100B1000EFF05FEE630C0500232C85028320C100FB
:100B20000324810013010101678000007370043009
:100B30006F000000130101FB23261104232481040C
:100B40002322910423202105232E3103232C41034A
:100B5000232A510323286103232671032326C1007E
:100B600063060528638C052693072000639CF60026
:100B70000327C503930710006306F7007370043062
:100B80006F0000001389060093840500130405001C
:100B9000EF300065631A05008327C10063860700F4
:100BA000737004306F000000EF305003032784039C
:100BB0008327C403130B0000930B20009309F0FF5D
:100BC000130A0401930A44026364F710630479234F
:100BD0008327C1006382073663160B00130581016A
:100BE000EF308049EF30D002EF10D074EF30007F4B
:100BF0008327440463943701232204048327840455
:100C00006394370123240404EF3090009305C1005E
:100C100013058101EF30404963160530EF30007C49
:100C2000032784038327C4036304F710EF30407E57
:100C3000EF30C07A832784046346F0026F0000031C
:100C400013850A00EF30802863040500EF3040551B
:100C5000832784049387F7FF2324F40483278404E1
:100C60006356F00083274402E39C07FC23243405E9
:100C7000EF30007AEF308076832744046346F00239
:100C80006F00000313050A00EF30402463040500E1
:100C9000EF300051832744049387F7FF2322F404A5
:100CA000832744046356F00083270401E39C07FC78
:100CB00023223405EF30C075EF20401B130B1000CA
:100CC000EF30C071032784038327C403E370F7F078
:100CD0000326040463040612631A091E0325840014
:100CE00093850400EF504007832784008326040483
:100CF00003274400B387D7002324F40063E4E710FC
:100D00008327840383260400032744029387170064
:100D10002324D400232CF40263000710130544029B
:100D2000EF30C01A930710006318F50E6F004014DF
:100D3000EF30006E8325C10013050A00EF20106C10
:100D4000EF30C069832784046346F0026F0000031C
:100D500013850A00EF30801763040500EF3040442C
:100D6000832784049387F7FF2324F40483278404D0
:100D70006356F00083274402E39C07FC23243405D8
:100D8000EF300069EF308065832744046346F0024A
:100D90006F00000313050A00EF30401363040500E1
:100DA000EF300040832744049387F7FF2322F404A5
:100DB000832744046356F00083270401E39C07FC67
:100DC00023223405EF30C064EF20400AE31805EE1B
:100DD000EFF00FFC130B10006FF09FEE832705045C
:100DE000E38407D8737004306F0000007370043020
:100DF0006F00000003260404631006088327040024
:100E0000638607048327840303274402938717001C
:100E1000232CF402E31407F0EF30805F1305100079
:100E20008320C10403248104832441040329010491
:100E30008329C103032A8103832A4103032B01036E
:100E4000832BC102130101056780000003254400C4
:100E5000EF30C04B8327840303274402232204007E
:100E600093871700232CF402E31A07EAE30605FA36
:100E7000EFF00FF26FF05FFA0325C40093850400D2
:100E8000EF40906D832704040327C40083260400E9
:100E9000B307F0403307F7002326E400637ED7044E
:100EA00003274400B307F7002326F40013072000AC
:100EB000832744026304E90403278403130717000C
:100EC000232CE402E38A07F46FF05FE50325C400F6
:100ED00093850400EF405068832704040327C4006F
:100EE00083260400B307F0403307F7002326E4000D
:100EF000E37ED7FA6FF0DFFA8327440203278403E7
:100F0000E30C07FA032784031307F7FF232CE402FB
:100F10000327840313071700232CE402E38E07EE54
:100F20006FF0DFDF13050400EFF05F92EF10107435
:100F3000130500006FF0DFEEEF30804D1305000069
:100F40006FF01FEE130101FF2322910093040500AF
:100F5000130540052324810023261100EF40503F54
:100F600013040500630C0504232C05029307F0FF0E
:100F70002322F5041307100013050501232EE402B4
:100F80002324F40423220400232004002324040047
:100F9000232604002320040423089404EFF00FF90F
:100FA00013054402EFF08FF89306000013060000CB
:100FB0009305000013050400EFF0DFB713050400EC
:100FC0008320C10003248100832441001301010117
:100FD0006780000063040504130101FF23248100DE
:100FE00023229100232611002320210103294500FB
:100FF00013040500EF30C01D930400006304A90230
:101000008320C1000324810013850400032901000B
:1010100083244100130101016780000073700430D4
:101020006F0000008327C400930410009387F7FF2C
:101030002326F400E39607FC930600001306000045
:101040009305000013050400EFF0DFAE6FF05FFBC7
:101050006302050A63880508130101FE232C810041
:10106000232A91002328210123244101232E11004A
:1010700023263101930720009384060013090600FC
:10108000138A050013040500639CF6000327C503BB
:10109000930710006302F70A737004306F000000BA
:1010A000EFF04FE3032784038327C403930905006C
:1010B0006366F7049304000013850900EFF00FE165
:1010C0008320C10103248101138504000329010148
:1010D000832441018329C100032A810013010102F5
:1010E0006780000083270504E38807F673700430E7
:1010F0006F000000737004306F00000003260404CA
:10110000631E060C8327040063860712832784036B
:101110001307F0FF93871700232CF402832784041E
:101120006388E70E832784049304100093871700D5
:101130002324F4046FF05FF8EFF0CFD90327840382
:101140008327C403930905006360F706032604049C
:10115000E30A06FA0325C40093050A00EF40D03FD6
:10116000832704040327C40083260400B307F04048
:101170003307F7002326E4006378D70003274400F1
:10118000B307F7002326F40093072000E390F4F858
:1011900083278403E38C07F6832784039387F7FF71
:1011A000232CF4026FF09FF603260404E30C06F4EC
:1011B0000325C40093050A00EF40103A8327040476
:1011C0000327C40083260400B307F0403307F70069
:1011D0002326E400E364D7FA6FF09FFBE39C04F658
:1011E0000325840093050A00EF401037832784000D
:1011F0008326040403274400B387D7002324F40084
:10120000E3E6E7F0832704002324F4006FF01FF0E7
:101210008327440293041000E38007EA1305440285
:10122000EF20D04AE30A05E8E30809E82320990003
:101230006FF09FE803254400EF30400D23220400A7
:101240006FF0DFEC6302050A83270504638607005D
:10125000737004306F00000083270500638A07085D
:10126000130101FE232C8100232A910013040500A1
:101270002328210123263101232E11001389050083
:10128000EFF04FC5032784038327C40393090500A8
:10129000930400006376F702832784031307F0FFAB
:1012A00093871700232CF40283278404638AE704BE
:1012B0008327840493041000938717002324F404E5
:1012C00013850900EFF08FC08320C1010324810141
:1012D0001385040003290101832441018329C100EE
:1012E0001301010267800000737004306F0000007A
:1012F00083274500E38607F6737004306F00000013
:101300008327440263960700930410006FF05FFB8D
:1013100013054402EF20903BE30805FEE30609FEB7
:10132000930710002320F9006FF01FFE130101FC4A
:10133000232E1102232C8102232A91022328210328
:101340002326310323244103232251032326C100F2
:1013500063060528638C0526938A06009389050099
:1013600013040500EF20D067631A05008327C1002E
:1013700063860700737004306F000000EF300006D2
:10138000832784036394071C8327C10063800710AD
:1013900013058101EF20504E9304F0FF130944021E
:1013A000130A0401EF30C006EF10C078EF300003DD
:1013B000832744046394970023220404832784042E
:1013C0006394970023240404EF3080049305C10044
:1013D00013058101EF20504D63100524EF3000000C
:1013E00083278403638A070AEF308002EF20107F8F
:1013F000832784046346F0026F000003130509008D
:10140000EF20D02C63040500EF209059832784043B
:101410009387F7FF2324F404832784046356F000A2
:1014200083274402E39C07FC23249404EF20507E8E
:10143000EF20D07A832744046346F0026F00000354
:1014400013050A00EF20902863040500EF20505593
:10145000832744049387F7FF2322F404832744045B
:101460006356F00083270401E39C07FC23229404C5
:10147000EF20107AEF10901FEF205076832784031F
:101480006396070C8327C100E39E07F0EF20507896
:10149000130500006F00800FEF2090778327040072
:1014A000638807108325C10013050900EF2000752C
:1014B000EF20D072832784046346F0026F0000039C
:1014C00013050900EF20902063040500EF20504D24
:1014D000832784049387F7FF2324F4048327840459
:1014E0006356F00083274402E39C07FC2324940402
:1014F000EF201072EF20906E832744046346F002C1
:101500006F00000313050A00EF20501C6304050060
:10151000EF201049832744049387F7FF2322F40424
:10152000832744046356F00083270401E39C07FCEF
:1015300023229404EF20D06DEF10501363040508AC
:10154000EF20D06983278403E38E07F29385090097
:10155000130504008324C400EFF00FAC63940A0861
:1015600083278403032704009387F7FF232CF402C7
:1015700063160700EF2010712322A40083270401C3
:1015800063920708EF20D068130510008320C10381
:101590000324810383244103032901038329C10216
:1015A000032A8102832A410213010104678000009B
:1015B000EF20D06203254400EF205045EF20506516
:1015C0006FF05FEEEFE0DFFC6FF09FF7832705041D
:1015D000E38407D8737004306F0000007370043028
:1015E0006F0000008327440223269400E38C07F851
:1015F00013054402EF20900DE30605F8EFE05FF9D4
:101600006FF05FF813050401EF20500C93071000F2
:10161000E31AF5F66FF09FFE13050400EFF00FA339
:10162000EF10D004130500006FF05FF663000506AD
:10163000130101FF2324810023202101232611000F
:10164000232291008324450013890500130405001B
:10165000EF2010386380A4049306000013060900ED
:101660009305000013050400EFF05FCC9307100012
:10167000630CF5028320C100032481008324410010
:101680000329010013010101678000007370043019
:101690006F0000008327C400130510009387170014
:1016A0002326F4006FF01FFD8327C40093871700E3
:1016B0002326F4006FF01FFC630805066386050C03
:1016C000130101FE232C8100232A910023282101EC
:1016D000232631012324410113040500232E110088
:1016E0001309060093890500EFE0DFFE83278403DA
:1016F000130A050093040000639C070213050A0007
:10170000EFE0DFFC8320C101032481011385040085
:1017100003290101832441018329C100032A810097
:101720001301010267800000737004306F00000035
:1017300003260404630406028325C40083274400AF
:10174000B385C5002326B40063E6F50083250400B5
:101750002326B40013850900EF400060832784032B
:101760001307F0FF9387F7FF232CF4028327440429
:101770006384E702832744049304100093871700CF
:101780002322F4046FF09FF783270504E38A07F20E
:10179000737004306F000000832704016396070014
:1017A000930410006FF09FF513050401EF20007201
:1017B000E30805FEE30609FE930710002320F90065
:1017C0006FF01FFE6306050883270504638A05087A
:1017D00063840708130101FE232C8100232A910052
:1017E000232821012324410113040500232E110085
:1017F00023263101138A0500EFE0DFED8327840300
:101800001309050093040000638E07008329C400B8
:1018100093050A0013050400EFF00F8093041000F5
:101820002326340113050900EFE05FEA8320C1019C
:10183000032481011385040003290101832441014C
:101840008329C100032A810013010102678000007F
:10185000737004306F000000737004306F0000007C
:10186000E38C07FE737004306F0000006316050000
:10187000737004306F000000130101FF2324810006
:101880001304050023261100EF20503503248403A0
:10189000EF2010388320C1001305040003248100C9
:1018A00013010101678000006316050073700430A6
:1018B0006F000000130101FF232611002324810083
:1018C00013040500EF209031832784030324C4030D
:1018D0003304F440EF20D033130504008320C1000B
:1018E00003248100130101016780000063060500E5
:1018F0000325850367800000737004306F000000CB
:1019000063080504978703009387C7E703A7470089
:101910006304E50403A7C7006302E50803A74701C2
:10192000630AE50603A7C7016302E50603A74702AA
:10193000630AE50403A7C7026302E50403A747039C
:10194000630AE50203A7C7036302E5026F4040385C
:10195000737004306F000000130700001317370086
:10196000B387E70023A007006F408036130770009D
:101970006FF0DFFE130760006FF05FFE130750008B
:101980006FF0DFFD130740006FF05FFD13073000BD
:101990006FF0DFFC130720006FF05FFC13071000EF
:1019A0006FF0DFFB0325C504678000002326B50424
:1019B0006780000003450505678000006308050097
:1019C000032585031335150067800000737004300C
:1019D0006F000000630C0500832785030325C50302
:1019E0003305F5401335150067800000737004302F
:1019F0006F000000978703009387C7D803A70700ED
:101A00006300070403A787006308070403A707010F
:101A10006308070403A787016308070403A70702F5
:101A20006308070403A787026308070403A70703E3
:101A3000630C070403A7870363040704678000009F
:101A40001307000013173700B387E70023A0B70080
:101A500023A2A70067800000130710006FF09FFE0D
:101A6000130720006FF01FFE130730006FF09FFD7B
:101A7000130740006FF01FFD130750006FF09FFC2D
:101A8000130770006FF01FFC130760006FF09FFBDF
:101A900097870300938707CF03A747006300E504F8
:101AA00003A7C7006306E50403A747016306E5042F
:101AB00003A7C7016306E50403A747026306E5041D
:101AC00003A7C7026306E50403A74703630AE50407
:101AD00003A7C7036302A704678000001307000081
:101AE00013173700B387E70023A0070067800000C3
:101AF000130710006FF0DFFE130720006FF05FFE8A
:101B0000130730006FF0DFFD130740006FF05FFD3B
:101B1000130750006FF0DFFC130770006FF05FFCDD
:101B2000130760006FF0DFFB130101FF2324810026
:101B300023229100232021011304050023261100F4
:101B40009384050013090600EF205009032744047D
:101B50009307F0FF6314F70023220404032784048F
:101B60009307F0FF6314F70023240404EF20500AC6
:101B700083278403639A07001306090093850400F2
:101B800013054402EF20C023EF205005832784046F
:101B9000635AF004832744026386070493044402D3
:101BA0006F000002832784049387F7FF2324F40443
:101BB000832784046358F002832744026384070266
:101BC00013850400EF208030E30E05FCEF20405D1C
:101BD000832784049387F7FF2324F4048327840452
:101BE000E34CF0FC9307F0FF2324F404EF205002B1
:101BF000EF20C07E83274404635AF0048327040146
:101C000063860704930404016F00000283274404E1
:101C10009387F7FF2322F404832744046358F002D8
:101C2000832704016384070213850400EF20002A40
:101C3000E30E05FCEF20C056832744049387F7FF8B
:101C40002322F40483274404E34CF0FC9307F0FFC1
:101C50002322F404032481008320C1008324410053
:101C600003290100130101016F20807A6304050438
:101C7000130101FD232E3101232C410123261102E2
:101C8000138A0700232481022322910223202103A7
:101C9000232A510123286101232671012324810174
:101CA000930790009309070063FAE700737004300C
:101CB0006F000000737004306F000000930A05008D
:101CC0009384050013090600938B0600130B08008C
:101CD0006304082C13050006EF3090671304050019
:101CE0006304052A13192900232865031306090034
:101CF0009305500A13050B00EF40001803C70400BA
:101D0000832704031309C9FF230AE40203C704005D
:101D1000338927011379C9FF6306070E83C71400AF
:101D2000A30AF40283C71400638E070C83C7240040
:101D3000230BF40283C724006386070C83C7340097
:101D4000A30BF40283C73400638E070A83C74400E1
:101D5000230CF40283C744006386070A83C7540038
:101D6000A30CF40283C75400638E070883C7640082
:101D7000230DF40283C764006386070883C77400D9
:101D8000A30DF40283C77400638E070683C7840023
:101D9000230EF40283C784006386070683C794007A
:101DA000A30EF40283C79400638E070483C7A400C4
:101DB000230FF40283C7A4006386070483C7B4001B
:101DC000A30FF40283C7B400638E070283C7C40065
:101DD0002300F40483C7C4006386070283C7D400CA
:101DE000A300F40483C7D400638E070083C7E40014
:101DF0002301F40483C7E4006386070083C7F4006B
:101E0000A301F404130B440013050B00A301040405
:101E10002326340323283405232A0404EFE01F93E8
:101E200013058401EFE09F929307A000B387374129
:101E3000232C040423288400232CF400232284026E
:101E400023220404232E040413860B0093850A0026
:101E500013050900EFE0DF882320A40063040A00D3
:101E600023208A007370043017E9010013094962C6
:101E70008327090097E4010093844463638C07007F
:101E800003A7040083A70400832747049387170050
:101E90002322F70417E70100130747608327070091
:101EA0009387170097E6010023AAF65E83A7040034
:101EB000638007108327090017EA0100130A4A709C
:101EC000639C070083A7040083A7C70263E6F900A9
:101ED00097E7010023AC875C97E701009387475A97
:101EE00003A7070097E601009386C65A8327C4021A
:101EF00083A606001307170017E601002322E65801
:101F00002324E40463F6F60017E701002324F758BE
:101F100013074001B387E70293050B003305FA006E
:101F2000EFE05F83832709006388070083A704002D
:101F300083A74704639E0708832709001304100042
:101F4000638A070083A7040083A7C70263F43701ED
:101F5000EFE00FE4130504008320C1020324810293
:101F600083244102032901028329C101032A81013B
:101F7000832A4101032B0101832BC100032C810023
:101F8000130101036780000013050B00EF3050546C
:101F90001304F0FF6FF01FFC13152600EF30503BC9
:101FA000130B0500E31805D21304F0FF6FF09FFA3E
:101FB00097E7010023AC874E032707009307100023
:101FC000630AF70217EA0100130A8A5F6FF0DFF075
:101FD00003A7040083A60400832747049387F7FF21
:101FE0002322F70483A74604E39807F473600430C0
:101FF0006FF09FF4930A000017EA0100130A4A5C8D
:10200000130C4001930BA00033858A03938A1A00B6
:102010003305AA00EFE08FF1E3987AFF97EB010018
:10202000938B8B6613850B00EFE04FF097EA01006E
:10203000938ACA6613850A00EFE04FEF17E50100A7
:1020400013050567EFE08FEE17E5010013058567BF
:10205000EFE0CFED17E5010013050568EFE00FEDA8
:1020600097E7010023A2774597E7010023AC574388
:102070006FF09FE6130101FF232481002326110046
:1020800023229100232021011304050073700430E2
:1020900097E401009384C43F83A70400639E071064
:1020A0006318040097E701009387474003A40700E3
:1020B0001309440013050900EFE00FF2832784029F
:1020C0006386070013058401EFE00FF19305090013
:1020D00017E501001305055FEFE0CFE797E7010083
:1020E0009387073C03A7070097E7010093874739C9
:1020F00083A707001307170097E6010023A2E63A1B
:1021000003A704009387170097E6010023AAF63679
:10211000630C070097E701009387473903A707007F
:1021200003274704631C070E83A70400638A07067E
:1021300097E701009387873703A70700630287109B
:102140007370043003A704006318070817E7010041
:10215000130787358326070083A606006392060AC5
:102160001307F0FF97E6010023AAE63003A7040057
:102170006308070203A70700032747046302070257
:1021800003A7070083A60700832747049387F7FF69
:102190002322F70483A74604639407007360043086
:1021A0008320C1000324810083244100032901000E
:1021B000130101016780000097E701009387072F53
:1021C00003A7070083A70700832747049387170007
:1021D0002322F7046FF0DFEC83A6070003A70700B4
:1021E00003A746041307170023A2E60417E701001C
:1021F0001307872B8326070083A60600E38206F6D3
:10220000032707000327C7000327C700032747004A
:1022100097E6010023A4E6266FF05FF503A7070009
:1022200083A60700832747049387F7FF2322F70439
:1022300083A74604E39A07EE736004306FF0DFEE85
:1022400097E701009387472383A70700638607006A
:10225000737004306F000000032481008320C100EC
:102260008324410003290100130101016FE04FB2F3
:102270006304050C17E701001307472383260700B3
:10228000930700006386A60A130101FF23261100AD
:1022900023248100232291007370043097E601000B
:1022A0009386061F83A70600638C0700032607009A
:1022B0008327070083274604938717002322F60409
:1022C00083A70600930405000324450163880700E3
:1022D0008327070083A747046394070697E7010055
:1022E0009387871C83A70700638C870697E7010005
:1022F0009387471B83A707006384870697E701003E
:102300009387873D6306F40497E701009387873B33
:10231000630CF402930710008320C10003248100A2
:102320008324410013850700130101016780000029
:102330001385070067800000737004306F00000091
:10234000EF60806C6FF09FF9930740006FF0DFFC47
:1023500083A7840293B71700938727006FF0DFFBF2
:10236000930720006FF05FFB7370043097E7010064
:102370009387071203A70700631607026304050487
:1023800083A707000325C502638C070097E70100B8
:102390009387C71103A7070003274704631C07029D
:1023A0006780000017E70100130747108326070026
:1023B0000327070003A746041307170023A2E60418
:1023C000E31005FC17E701001307470E032507007C
:1023D0006FF01FFB03A7070083A6070083274704AE
:1023E0009387F7FF2322F70483A74604E39A07FAAB
:1023F0007360043067800000130101FF2324810013
:102400001304050023261100EFE0CFAC631804008D
:1024100097E701009387870903A407000324C402F8
:10242000EFE0CFAA8320C10013050400032481003C
:1024300013010101678000009307900063F6B70065
:10244000737004306F000000130101FE232C810023
:10245000232E1100232A9100232821012326310154
:1024600023244101130405007370043017E90100AF
:1024700013090902832709006392071063000412FD
:1024800083270405638EF50A17E701001307070287
:1024900063F0B70283260700638E861203270700C6
:1024A0008324C702B3B4950093C414006F000001E5
:1024B00083240700B384844093B414000327C40228
:1024C0006386E70E832784012328B40463C80700CA
:1024D0009307A000B385B740232CB40093172700BF
:1024E000B387E7000327440197E901009389490D69
:1024F00093972700B387F9006310F704130A440089
:1025000013050A00EFE04FAD17E70100130787F846
:102510008327C402032707006376F70017E701004B
:10252000232AF7F613074001B387E70293050A0051
:102530003385F900EFE00FA263840400EFE04F85DC
:1025400083270900638C070097E70100938707F64C
:1025500083A7070083A74704639E07048320C10164
:102560000324810183244101032901018329C1003E
:10257000032A8100130101026780000097E7010030
:102580009387C7F203A7070083A7070083274704A1
:10259000938717002322F704E31404EE97E7010062
:1025A0009387C7F003A407006FF09FED2326B402C2
:1025B0006FF05FF1032481018320C1018324410175
:1025C000032901018329C100032A810013010102AB
:1025D0006F608043930400006FF05FEE630A0508AC
:1025E000130101FE232A910097E40100938404EC77
:1025F00083A70400232E1100232C8100232821010E
:10260000232631016388A7047370043017E90100A1
:10261000130909E883270900638C070003A7040056
:1026200083A7040083274704938717002322F70416
:102630000327450197E701009387070A630EF70216
:10264000832709006388070083A7040083A7470442
:10265000639E07088320C101032481018324410173
:10266000032901018329C1001301010267800000D1
:10267000737004306F0000008327850217E70100A4
:1026800013070703E38EE7FAE39C07FA9309450073
:102690001304050013850900EFE00F9417E701000C
:1026A000130747DF8327C402032707006376F70079
:1026B00017E701002320F7DE13074001B387E70285
:1026C00017E501001305C5EF938509003305F500F3
:1026D000EFE04F8883A704000327C40283A7C70243
:1026E000E360F7F6EFD0DFEA6FF09FF50324810196
:1026F0008320C10183244101032901018329C100F1
:10270000130101026F60403063020506130101FEF0
:10271000232C8100232A9100232821011304050082
:10272000232E110023263101EFD0DFFA03274401C5
:1027300097E70100938747FA130905009304000007
:10274000630AF70213050900EFD05FF88320C10187
:10275000032481011385040003290101832441011D
:102760008329C100130101026780000073700430E7
:102770006F0000008327840217E50100130545F36D
:10278000E382A7FCE39007FC97E701009387C7CE9D
:1027900083A707006394070697E70100938707D193
:1027A00083A707008324C4029309440083A7C702B8
:1027B00013850900B3B4F400EFE00F8217E70100BE
:1027C000130747CD8327C4020327070093C41400CF
:1027D0006376F70017E70100232EF7CA13074001BD
:1027E000B387E70217E50100130585DD938509002E
:1027F0003305F500EFD01FF66FF0DFF49305840189
:10280000EFD05FF56FF01FF4130101FE37150000E4
:10281000232E1100232C8100232A9100232821013B
:102820002326310123244101232251012320610168
:10283000EF300032630805229304050013050006FB
:10284000EF3000311304050063040526371600003D
:102850009305500A2328950213850400EF30C061C8
:1028600083240403B71700009387C7FFB384F400E1
:10287000B7474C4593879744130A4400232AF40230
:1028800013050A00230C0402A301040423260402F6
:1028900023280404232A0404EFD05FEB13058401EA
:1028A000EFD0DFEA9307A000232C040493F4C4FFC5
:1028B00023288400232CF4002322840223220404EE
:1028C000232E040413060000971500009385C5EA23
:1028D00013850400EFD0DFE02320A40073700430E0
:1028E00017E901001309C9BA8327090097E4010019
:1028F0009384C4BB638C070003A7040083A7040070
:1029000083274704938717002322F70417E7010062
:102910001307C7B8832707009387170097E60100BE
:1029200023AEF6B683A704006388070A832709004D
:1029300097E901009389C9C8639C070083A7040035
:1029400083A7C7026396070097E7010023A087B615
:1029500097E701009387C7B203A7070097E6010036
:10296000938646B38327C40283A606001307170085
:1029700017E601002326E6B02324E40463F6F600FC
:1029800017E701002328F7B0139527003305F5005A
:102990001315250093050A003385A900EFD09FDBAE
:1029A000832709006388070083A7040083A74704DF
:1029B000639E070C832709006384070083A7040034
:1029C000EF20100893071000630AF510631C050838
:1029D000737004306F00000097E7010023A887ACF4
:1029E000032707009307100097E90100938949BD69
:1029F000E310F7F6938A090017EB0100130BCBC81D
:102A000013850A00938A4A01EFD05FD2E31A5BFF75
:102A100017E50100130545C7EFD05FD197EA010024
:102A2000938ACAC713850A00EFD05FD017E501006B
:102A3000130505C8EFD09FCF17E50100130585C822
:102A4000EFD0DFCE17E50100130505C9EFD01FCE8B
:102A500097E7010023AA67A597E7010023A457A5DC
:102A60006FF01FEF8320C101032481018324410102
:102A7000032901018329C100032A8100832A41001F
:102A8000032B0100130101026780000003A704006B
:102A900083A60400832747049387F7FF2322F704C4
:102AA00083A74604E39807F0736004306FF09FF04B
:102AB000032481018320C101032901018329C1006D
:102AC000032A8100832A4100032B0100138504009F
:102AD00083244101130101026F30801F73700430A1
:102AE0009307F0FF17E70100232AF79803248101D9
:102AF00097E7010023AEA7988320C10183244101F9
:102B0000032901018329C100032A8100832A41008E
:102B1000032B010097E7010023A00798130101028E
:102B20006FD05F8C7370043097E7010023A2079683
:102B30006FD09F9D17E701001307079483270700B5
:102B4000938717002320F70067800000737004301C
:102B500097E701009387C79303A70700631807024D
:102B600017E70100130747930325070083A7070012
:102B7000638C070097E701009387479303A707003B
:102B800003274704631407026780000017E701006A
:102B90001307C791832607000327070003A74604EE
:102BA0001307170023A2E6046FF09FFB03A707009B
:102BB00083A60700832747049387F7FF2322F704A0
:102BC00083A74604E39207FC73600430678000002B
:102BD000130101FF2326110023248100EFD09FAFB2
:102BE00097E701009387478B03A40700EFD01FAE40
:102BF0008320C10013050400032481001301010197
:102C00006780000097E701009387478903A50700C5
:102C100067800000130101FD232611022324810295
:102C20002322910223202103232E3101232C410151
:102C3000232A5101232861012326710197E701000E
:102C40009387878383A70700639A070617E7010026
:102C500013078784832707009387170097E60100EF
:102C600023ACF682832A0700638A0A0A97E70100E9
:102C70009387C78083A707009304000063FEFA0AC6
:102C800097E901009389C99317EA0100130A0A82A0
:102C900083270A009306100003A7C7029317270093
:102CA000B387E70093972700B389F90083A709004A
:102CB00063F4F602930410006F00000297D701003E
:102CC0009387C77C83A707009304000093871700AE
:102CD00017D70100232CF77A97D701009387C77A7B
:102CE00083A7070063840700930410008320C102B8
:102CF0000324810213850400032901028324410275
:102D00008329C101032A8101832A4101032B010187
:102D1000832BC100130101036780000017D4010059
:102D2000130484788327040083A707006388070CB3
:102D3000737004306F00000017D401001304C476D0
:102D400097E901009389C98717DA0100130A0A7607
:102D500017DB0100130B0B748327040083A7070004
:102D6000638007088327040083A7C70003A9C7005F
:102D700083274900930B490013850B0063EAFA0689
:102D8000EFD09FA58327890213058901638407007B
:102D9000EFD09FA48327C90203270B0093850B0064
:102DA000139527003305F500131525003385A90079
:102DB0006376F70017D70100232EF76CEFD09F99A9
:102DC00083270A000327C90283A7C702E366F7F82F
:102DD000832704009304100083A70700E39407F8F7
:102DE0009307F0FF17D70100232AF7686FF05FEA17
:102DF00017D701002324F7686FF09FE917D7010068
:102E00001307476A832704000327070097D60100AA
:102E100023ACE66817D701002326F76897D701008F
:102E20009387476683A707009387170017D701008A
:102E3000232AF7648327040083A70700639A070007
:102E40009307F0FF17D70100232AF7626FF01FE204
:102E50008327040083A7C70083A7C70083A7470071
:102E600017D70100232CF7606FF05FE097D70100C0
:102E70009387876003A70700631607007370043009
:102E80006F000000130101FE232E1100232C81008E
:102E9000232A9100232821012326310123244101E3
:102EA00023225101232061017370043097D4010063
:102EB0009384045E03A704006310071203A70700AE
:102EC0001307F7FF97D6010023A8E65A83A7070048
:102ED000639E070A97D701009387475C83A7070083
:102EE0006386070A97DA0100938A8A6D17DA010070
:102EF000130A4A5A17D901001309495B93091000B4
:102F00006F00C0013385EA00EFD0DF84832709001A
:102F10000327C40283A7C7026374F70683A70A0FB7
:102F20006380070E83A7CA0F03A4C700130584019B
:102F3000EFD09F8A130B440013050B00EFD0DF89FD
:102F40008327C40283260A0093050B0013952700EC
:102F50003305F50013152500130705003385AA0076
:102F6000E3F2F6FA17D701002326F752EFD08FFECF
:102F7000832709000327C40283A7C702E360F7FA87
:102F800097D7010023A237516FF05FF913040000B7
:102F900083A70400638C070097D70100938707512C
:102FA00083A7070083A74704639807041305040059
:102FB0008320C101032481018324410103290101EC
:102FC0008329C100032A8100832A4100032B0100C9
:102FD000130101026780000017D701001307074D96
:102FE000832607000327070003A7460413071700DB
:102FF00023A2E6046FF09FECEF5010216FF01FFB4F
:1030000017D401001304844883270400638C07024B
:10301000832704001309100063860702EFF09FBFA7
:103020006306050097D7010023A0274783270400E4
:103030009387F7FF17D70100232AF744832704005B
:10304000E39E07FC97D701009387074403A7070077
:1030500093071000E31CF7F2EFD08FD31304100096
:103060006FF01FF36304050263960500737004306C
:103070006F00000017D701001307074083270700E0
:10308000638A0700737004306F00000073700430AF
:103090006F000000130101FF23248100232611008B
:1030A00083260700032705009386160017D6010024
:1030B0002324D63C97D601009386063E83A60600BD
:1030C0003304B7002320850063F0E6046372E40252
:1030D00063F0860297D701009387473D03A5070059
:1030E00013054500EFD04FEF13050400EF505009D2
:1030F000EFF0DFD7630E05008320C10003248100B9
:103100001301010167800000E366E4FC6FF05FFCDF
:10311000032481008320C100130101016FD04FC738
:10312000630E050017D70100130707358327070033
:1031300063880700737004306F0000006FD04FC5C4
:10314000130101FF23261100232481000327070018
:10315000930705001307170097D6010023AEE6304A
:1031600097D601009386863417D701001307C7321C
:103170000327070003A506003304F70013054500E5
:10318000EFD08FE513050400EF50807FEFF01FCEE6
:10319000631A0500032481008320C100130101018B
:1031A0006FD00FBF8320C1000324810013010101F0
:1031B00067800000130101FF2324810023261100F2
:1031C00097D701009387472B83A7070013040000BC
:1031D0009387170017D701002320F72A97D70100FC
:1031E0009387C72B83A7070063EEF51417DE010052
:1031F000130ECE4897D201009382C23B1304000005
:1032000013070000930F10001303500A6F00C00053
:10321000130ECEFE6384C20F83278EFF9306070032
:10322000E38807FE8327CEFF83A74700232EFEFEF9
:103230006386C71303AFC70083A747003307E500C2
:10324000930E0000232EFEFE6380C70983A8C700EB
:1032500093874803232017012322F70083A78804BC
:103260002326F7012324F70083A7C8022328F700A9
:1032700083A70805232C0700232AF70003A80803C7
:103280008347080063986704930708009387170033
:1032900083C60700B3850741E38A66FE93D5250000
:1032A0009395050193D50501231EB700938E1E004B
:1032B00013070702630A1F038327CEFF83A7470074
:1032C000232EFEFEE394C7F983274E00232EFEFE35
:1032D0006FF0DFF793050000231EB700938E1E00EA
:1032E00013070702E31A1FFD3304D4011317540018
:1032F000130ECEFE93060700E390C2F397D70100AA
:103300009387871A03AE070083270E006396071280
:1033100097D701009387071903AE070083270E0094
:10332000639A071C17DE0100130E8E2983274E10A7
:10333000639C070283278E11639C072663040600A3
:1033400023200600EFF09FB2130504008320C10084
:1033500003248100130101016780000083274E00D0
:10336000232EFEFE6FF01FED83278E1017DF010066
:10337000130FCF3583A7470017D701002326F73453
:103380006386E73D83A2C70083A74700B306D50045
:10339000930E000017D701002328F732930F400047
:1033A0001303500A6382E70983A8C7009387480381
:1033B00023A0160123A2F60083A7880423A6F60102
:1033C00023A4F60083A7C80223A8F60083A7080554
:1033D00023AC060023AAF60003A8080383470800CD
:1033E000639A6732930708009387170003C70700A3
:1033F000B3850741E30A67FE93D72500939707013A
:1034000093D70701239EF600938E1E009386060233
:10341000638C123183278E1083A7470017D70100D2
:103420002324F72AE392E7F983270E1117D7010027
:10343000232CF7286FF05FF783274E00130F8E00C1
:1034400083A647002322DE006380E633B307E5004E
:1034500003A7460083A2C600930E00002322EE00BD
:10346000930F20001303500A6300EF088328C7005E
:103470001387480323A0170123A2E70003A78804AA
:1034800023A6F70123A4E70003A7C80223A8E700A7
:1034900003A7080523AC070023AAE70003A8080335
:1034A00003470800631E672213070800130717006D
:1034B00083460700B3050741E38A66FE13D725005C
:1034C0001317070113570701239EE700938E1E0071
:1034D000938707026380122383264E0003A74600CA
:1034E0002322EE00E314EFF80327CE002322EE00A0
:1034F0006FF0DFF783274E00130F8E0083A747007E
:103500002322FE00638CE72583A2C70083A7470020
:10351000B306D500930E00002322FE00930F200077
:103520001303500A6300FF0883A8C700938748036A
:1035300023A0160123A2F60083A7880423A6F60180
:1035400023A4F60083A7C80223A8F60083A70805D2
:1035500023AC060023AAF60003A80803834708004B
:1035600063986714930708009387170003C7070041
:10357000B3850741E30A67FE93D7250093970701B8
:1035800093D70701239EF600938E1E0093860602B2
:10359000638A121383274E0083A747002322FE006D
:1035A000E314FFF88327CE002322FE006FF0DFF73D
:1035B0008327CE1197DE0100938E8E1283A74700DA
:1035C00017D70100232CF710638AD71783AFC700E2
:1035D00083A747003307D5001303000097D60100E7
:1035E00023AEF60E130F3000930220009308500A0A
:1035F0006388D70903A5C700930745032320A700C5
:103600002322F700832785042326E7012324F700DC
:103610008327C5022328F7008327850263840700D8
:103620002326570083270505232C0700232AF700AC
:103630000328050383470800639C170593070800C8
:103640009387170083C60700B3850741E38A16FFF7
:1036500093D725009397070193D70701231EF700FF
:103660001303130013070702638EAF028327CE11E3
:1036700083A7470097D6010023A2F606E39CD7F75D
:1036800083274E1297D6010023AAF6046FF09FF607
:1036900093070000231EF70013031300130707020C
:1036A000E396AFFC33046400E31C06C86FF09FC9C7
:1036B00093070000239EF600938E1E009386060259
:1036C000E39A12ED17DE0100130E8EEF83274E10E2
:1036D0003304D40193165400E38E07C46FF0DFC89F
:1036E00013070000239EE700938E1E0093870702B6
:1036F000E39412DF97D701009387C7DA03AE070080
:103700003304D4019316540083270E00E38C07C0C2
:103710006FF05FDE93070000239EF600938E1E007D
:1037200093860602E39812CF83278E113304D401C7
:1037300093165400E38407C06FF09FE783274E126F
:1037400017D70100232CF7F86FF05FE883270E11DD
:1037500017D70100232AF7F66FF0DFC28327CE00C8
:103760002322FE006FF05FDA8326CE002322DE00E4
:103770006FF0DFCD130101FD2322910223202103ED
:10378000232E3101232C4101232A510123286101D9
:1037900023267101232611022324810297D90100D7
:1037A000938989CD17D90100130989E117DA01003E
:1037B000130A0ACE97DA0100938A4ACF97DB0100F9
:1037C000938BCBCD97D40100938484CD130B100041
:1037D0006F00000283A70900032449109387170094
:1037E00017D70100232AF7C8EFF04FE8631E040043
:1037F00083A70400E39007FE83270900E37AFBFE1A
:10380000EFC01FD96FF0DFFE7370043083270A000A
:10381000639E07048327091103A4C700130544000E
:10382000EFC09FFB83A70B009387F7FF17D701001B
:103830002326F7C683A704009387F7FF17D7010055
:103840002320F7C683270A006388070083A70A009E
:1038500083A747046398070203250403EF2040472A
:1038600013050400EF20C0466FF09FF803A70A007D
:1038700083A70A0083274704938717002322F704AE
:103880006FF05FF903A70A0083A60A0083274704A5
:103890009387F7FF2322F70483A74604E39E07FAE2
:1038A000736004306FF05FFB97D701009387C7BC4C
:1038B00083A707006396070E130101FF232611005B
:1038C00097D7010023A207BC17D70100130707BE33
:1038D00083270700B7A6A5A59386565A83A7070393
:1038E00083A50700639ED50003A64700631AB600B0
:1038F00083A687006396C60083A7C700638AD700A4
:10390000032507008325070093854503EF30D00D7D
:1039100097D60100938606B803A6060017D70100C4
:10392000130707CA6F00000283A706006382070817
:1039300083A706009387F7FF17D60100232CF6B460
:1039400003A6060093172600B387C70093972700A6
:10395000B307F70083A70700E38807FC03A6060068
:1039600093172600B387C70093972700B305F70086
:1039700083A6450093878700B307F70083A6460018
:1039800023A2D500638AF60283A7C6008320C10064
:1039900017D70100232CF7B0130101016780000045
:1039A0009307100017D701002320F7AE67800000AF
:1039B000737004306F000000930740013306F60275
:1039C00083A646003307C7002322D7006FF0DFFB32
:1039D000130101FE23282101232E1100232C810035
:1039E000232A910023263101130905007370043046
:1039F00097D401009384C4A983A7040017D40100BD
:103A00001304C4AA639C070C63140900032904006F
:103A10009309490013850900EFC01FDC8327890241
:103A20006386070013058901EFC01FDB938509003A
:103A300017D50100130545CAEFC0DFD183A70400E5
:103A4000638807008327040083A747046394070A59
:103A5000832704006384270D83A70400638207067D
:103A60007370043083A704006398070E97D7010092
:103A7000938787A303A70700032707006310070C9A
:103A80009307F0FF17D70100232AF79E83A70400AE
:103A9000638807028327040083A747046382070221
:103AA0000327040083260400832747049387F7FF36
:103AB0002322F70483A7460463940700736004304D
:103AC0008320C101032481018324410103290101D1
:103AD0008329C1001301010267800000032704004D
:103AE0008327040083274704938717002322F704C2
:103AF0006FF09FF103270400832604008327470407
:103B00009387F7FF2322F70483A74604E39207F481
:103B10007360043083270400E39027F583A7040033
:103B20006382070697D701009387079583A707004D
:103B30006388070A737004306F00000083A70700D2
:103B400083A7C70083A7C70083A7470017D7010033
:103B50002326F7926FF09FF30327040083270400C6
:103B600083274704938717002322F70497D7010080
:103B70009387879303A7070003270700E30207F053
:103B80006FF0DFFB97D701009387479117D70100AC
:103B9000130707A383A70700032787116314F702FE
:103BA0008320C1010324810197D7010023A007903E
:103BB00083244101032901018329C100130101026A
:103BC00067800000032481018320C1018324410117
:103BD000032901018329C100130101026FF0DFCC29
:103BE000032481018320C1018324410103290101B0
:103BF0008329C100130101026FC09F996306050A62
:103C0000130101FF2322910097D401009384048AB9
:103C1000232021011389050083A504002326110018
:103C20002324810093858501EFC0DFB503A504003F
:103C300013054500EFC05FBA9307F0FF630AF9066A
:103C400097D701009387478503A4070003A70400C3
:103C500083A707003304240123228700636EF40640
:103C600097D701009387478403A5070083A5040025
:103C700093854500EFC01FB197D701009387078058
:103C800083A707006376F40097C7010023A8877E07
:103C90008320C10003248100832441000329010003
:103CA0001301010167800000737004306F00000091
:103CB00083A50400032481008320C10083244100E4
:103CC0000329010017D50100130505A193854500BF
:103CD000130101016FC01FA897C701009387877C5C
:103CE00003A507000324810083A504008320C100ED
:103CF000832441000329010093854500130101013C
:103D00006FC05FA8630E050097C701009387C77651
:103D100083A70700639A0700737004306F000000E8
:103D2000737004306F000000130101FF2322910023
:103D300097C401009384847703A704009387050048
:103D400083A50400B7060080B3E7D700232611003F
:103D500023248100232CF70093858501130406009A
:103D6000EFC05F9F03A5040013054500EFC0DFA669
:103D70009307F0FF6304F40297C701009387C771AC
:103D800003A507008320C10083244100330585007B
:103D900003248100130101016F40903E83A50400BC
:103DA000032481008320C1008324410017D5010032
:103DB0001305859293854500130101016FC09F99FA
:103DC0006308050A130101FF2322910097C4010033
:103DD0009384C46D232021011389050083A5040069
:103DE00023261100232481009385850113040600F6
:103DF000EFC05F9603A5040013054500EFC0DF9DEB
:103E000093071000630AF40697C701009387C768F9
:103E100003A4070003A7040083A7070033042401B9
:103E200023228700636EF40697C701009387C76754
:103E300003A5070083A5040093854500EFC09F9468
:103E400097C701009387876383A707006376F40011
:103E500097C7010023A487628320C1000324810047
:103E60008324410003290100130101016780000040
:103E7000737004306F00000083A5040003248100E8
:103E80008320C100832441000329010017D50100CC
:103E90001305858493854500130101016FC09F8B35
:103EA00097C701009387076003A5070003248100DB
:103EB00083A504008320C10083244100032901005D
:103EC00093854500130101016FC0DF8B130101FFD2
:103ED0002326110023248100232291008327C5007B
:103EE00003A4C7006304040A930484011385040037
:103EF000EFC09F8E97C701009387075883A70700DD
:103F0000639A07089304440013850400EFC0DF8C14
:103F100097C70100938707580327C40283A70700A8
:103F200063F6E70097C7010023A6E756931727001B
:103F3000B387E7009397270017C50100130545686D
:103F4000938504003305F500EFC0DF8097C70100BB
:103F50009387C75583A707000327C40213050000F2
:103F600083A7C70263FAE7009307100017C7010091
:103F7000232CF750130510008320C1000324810077
:103F80008324410013010101678000007370043035
:103F90006F0000009385040017C5010013054571EB
:103FA000EFC04FFB6FF09FFA97C701009387C74C94
:103FB00083A7070063960700737004306F0000004A
:103FC000130101FF232611002324810023229100E5
:103FD000B70700800324C500B3E7F5002320F500F0
:103FE00063080408EFC04FFF9304440013850400E6
:103FF000EFC08FFE97C701009387C7490327C4020C
:1040000083A7070063F6E70097C7010023A4E748EA
:1040100093172700B387E7009397270017C5010080
:104020001305055A3305F50093850400EFC08FF2A0
:1040300097C701009387874783A707000327C40218
:104040001305000083A7C70263FAE7009307100077
:1040500017C70100232AF742130510008320C1006F
:1040600003248100832441001301010167800000C3
:10407000737004306F0000006304050297C70100ED
:104080009387474003A7070097C701009387C7405E
:1040900083A707002320E5002322F50067800000A6
:1040A000737004306F0000006304050E638E050C0E
:1040B000130101FF232611002324810013070500AB
:1040C0007370043097C801009388883C83A7080068
:1040D0006380070297C701009387473D83A60700C7
:1040E00083A7070083A746049387170023A2F6043B
:1040F00017C301001303433A83A7050003260300F7
:104100009306F0FF130400006388D70417CE010064
:10411000130E4E3703250E000328070083264700A1
:104120006306A800130410006378D6023308D64053
:10413000130410006372F80203250E00B387C74012
:1041400003260300B387D70023A0F5002320A70090
:104150002322C7001304000083A70800638C070014
:1041600097C701009387873483A7070083A7470475
:1041700063940702130504008320C1000324810017
:104180001301010167800000737004306F000000AC
:10419000737004306F000000EF4010076FF09FFD58
:1041A0009307100017C701002320F72E6780000037
:1041B000630605000325C5046780000013050000A1
:1041C00067800000630405002326B50467800000B3
:1041D00097C701009387872D03A50700678000001C
:1041E00097C701009387C72A83A70700130510000C
:1041F000638C070097C701009387072803A5070072
:10420000133515001315150067800000630C0508B1
:10421000130101FE232A910097C40100938404290D
:1042200083A70400232E1100232C810023282101C1
:10423000232631010327C50283A7C7026376F7044B
:104240008327850163CC070083A7040083A6C702E8
:104250009307A000B387D740232CF50093172700BE
:10426000B387E7000327450117C901001309493542
:1042700093972700B307F9006308F70283A70400A8
:1042800083A7C7022326F5028320C10103248101ED
:1042900083244101032901018329C1001301010283
:1042A0006780000067800000930945001304050043
:1042B00013850900EFC04FD283A7040017C7010080
:1042C0001307471D0327070083A7C7022326F4020D
:1042D0006376F70017C70100232EF71A13952700FE
:1042E0003305F50003248101131525008320C10146
:1042F00083244101938509003305A9008329C10066
:1043000003290101130101026FC0CFC46306050236
:10431000130101FF23261100232481002322910091
:1043200097C701009387871803A40700630AA400B6
:10433000737004306F0000001305000067800000F8
:104340008327440563960700737004306F000000F4
:104350008326C402032704059387F7FF232AF40466
:104360006384E600638E0700130500008320C1000C
:1043700003248100832441001301010167800000B0
:104380009304440013850400EFC00FC58327040580
:1043900017C7010013070710832607001307A000A3
:1043A0003307F7402326F402232CE40063F6F600DB
:1043B00017C701002320F70E13074001B387E70258
:1043C00017C501001305C51F938504003305F500CB
:1043D000EFC04FB8130510006FF05FF97370043031
:1043E00097C701009387C70A83A707006380070266
:1043F00097C701009387870B03A7070083A70700D0
:1044000083274704938717002322F704678000005F
:1044100097C701009387C70783A70700638C07022C
:1044200097C701009387870803A70700032747045E
:104430006302070203A7070083A607008327470438
:104440009387F7FF2322F70483A7460463940700AA
:10445000736004306780000097C7010093870705E9
:1044600003A6070083A6070003A707009307A00081
:1044700083A6C60203258601B387D740232CF70005
:104480006780000097C701009387470203A70700D2
:10449000630A070083A6070003A746051307170052
:1044A00023AAE60403A5070067800000130101FDAD
:1044B0002320210323261102232481022322910297
:1044C000232E3101130905007370043097C40100D5
:1044D000938404FC83A7040017C40100130404FDA3
:1044E000639E070A8327040083A78705639A070052
:1044F000832704001307100023AEE704639A050E18
:1045000083A70400638807008327040083A7470468
:10451000639A07147370043083A70400639407063A
:104520008327040003A587056308050063020904C7
:104530008327040023AC07048327040023AE070469
:1045400083A70400638807008327040083A7470428
:10455000639207068320C10203248102832441025F
:10456000032901028329C1011301010367800000AF
:1045700003270400832787059387F7FF232CF7047D
:104580006FF09FFB03270400832704008327470461
:10459000938717002322F7046FF09FF80327040086
:1045A0008327040083274704938717002322F704F7
:1045B0006FF05FF30327040083260400832747047A
:1045C0009387F7FF2322F70483A74604E39407F8B1
:1045D000736004308320C1020324810283244102DA
:1045E000032901028329C10113010103678000002F
:1045F000032504002326B10013054500EFC0CF9D1D
:104600008325C1009307F0FF6380F50897C7010079
:10461000938787E883A907000327040083A707007F
:10462000B389B9002322370163ECF90697C701006B
:10463000938787E703A5070083250400938545003A
:10464000EFC04F9497C70100938747E383A7070004
:1046500063F6F90097C7010023A237E3EFB05FF3D9
:104660006FF01FEA03270400832604008327470412
:104670009387F7FF2322F70483A74604E39C07E808
:10468000736004306FF01FE98325040017C5010033
:104690001305850493854500EFC0CF8B6FF01FFC99
:1046A00097C70100938707E003A50700832504004F
:1046B00093854500EFC00F8D6FF05FFA130101FD88
:1046C00023202103232E31012326110223248102DA
:1046D00023229102232C410113890500930906002E
:1046E0007370043097C40100938484DA83A70400B4
:1046F00017C40100130484DB639C07140327040020
:10470000930720000327C7056304F70283270400EB
:104710001345F5FF03A787053375E50023ACA70410
:10472000832704001307100023AEE704639A060AE8
:1047300083A70400638807008327040083A7470436
:10474000639407167370043083A70400639E070602
:10475000638809008327040083A7870523A0F90045
:104760000327040093071000130500000327C70563
:10477000630EF700832704001349F9FF13051000A7
:1047800003A787053379E90023AC270583270400B5
:1047900023AE070483A7040063880700832704006F
:1047A00083A747046392070C8320C102032481027C
:1047B00083244102032901028329C101032A8101C3
:1047C000130101036780000003270400832704000E
:1047D00083274704938717002322F7046FF05FF7BE
:1047E000032504002326D10013054500EFB0DFFEAA
:1047F0008326C1009307F0FF638AF60C97C7010078
:10480000938787C903AA07000327040083A707002B
:10481000330ADA00232247016368FA0C97C70100C4
:10482000938787C803A50700832504009385450067
:10483000EFB05FF597C70100938747C483A70700D0
:104840006370FA0A97C7010023AA47C36F004009A3
:104850000327040083270400832747049387170056
:104860002322F7046FF09FE9032704008326040046
:10487000832747049387F7FF2322F70483A746047F
:10488000E39407F2736004308320C10203248102A1
:1048900083244102032901028329C101032A8101E2
:1048A000130101036780000003270400832604002E
:1048B000832747049387F7FF2322F70483A746043F
:1048C000E39207E8736004306FF0DFE783250400AC
:1048D00017C50100130545E093854500EFB09FE73C
:1048E000EFB01FCB6FF0DFE497C70100938787BB62
:1048F00003A507008325040093854500EFB09FE8DA
:104900006FF01FFE630A050C130101FF232611003F
:10491000232481002322910023202101737004307D
:1049200097C401009384C4B683A704006396070864
:10493000638606008327850523A0F60093070600FB
:10494000930620000326C505232ED50413870500F2
:10495000130405006382D70A63F4F6089305300058
:104960006388B700930540006396B700630CD610C8
:10497000232CE40493071000630CF60813041000C2
:1049800083A70400638C070097C70100938707B2D1
:1049900083A7070083A7470463980706130504004D
:1049A0008320C100032481008324410003290100E6
:1049B000130101016780000097C70100938707AFCB
:1049C00003A7070083A707008327470493871700DF
:1049D0002322F7046FF0DFF5737004306F000000DE
:1049E00093061000E398D7F88327850533E7B700CF
:1049F000232CE5046FF01FF88327850593871700A4
:104A0000232CF5046FF01FF7EF4000006FF01FF943
:104A10001309440013050900EFB01FDC17C701009C
:104A2000130747A78327C402032707006376F7000D
:104A300017C701002320F7A613074001B387E70239
:104A400017C501001305C5B7930509003305F50027
:104A5000EFB05FD083278402638607007370043051
:104A60006F00000097C70100938747A483A7070042
:104A70000327C40283A7C702E3F2E7F0EFB05FB1F8
:104A80006FF0DFEF130400006FF09FEF630805087D
:104A9000130101FE232C8100232A910023282101E8
:104AA000232631012324410123225101232E110009
:104AB00093090700138A0600930406001389050072
:104AC00013040500EFB01FC1930A050063060A0036
:104AD000832784052320FA000327C40593072000B9
:104AE000232EF4046380F40463FA971093063000D5
:104AF0006388D400930640006396D400630CF70EDD
:104B0000232C2405930710006312F70A83278402DD
:104B100063820702737004306F000000737004300A
:104B20006F0000008327840593871700232CF4046B
:104B30006FF05FFD97C701009387079483A7070075
:104B40006390070A9304440013850400EFB0DFC8A4
:104B500017C70100130707948327C4020327070020
:104B60006376F70017C701002326F7921307400169
:104B7000B387E70217C50100130585A493850400D8
:104B80003305F500EFB01FBD97C70100938707926B
:104B900083A707000327C40283A7C70263F8E700BF
:104BA000638609009307100023A0F9001304100086
:104BB00013850A00EFB09FB1130504008320C101E3
:104BC0000324810183244101032901018329C100B8
:104BD000032A8100832A410013010102678000003B
:104BE0009305840117C50100130585ACEFB09FB68E
:104BF0006FF09FF9130400006FF09FFB9307100004
:104C0000E392F4F08327840533E92701232C24055C
:104C10006FF05FEF630A050E130101FE232C810084
:104C2000232A91001304050023282101232E1100BB
:104C30002326310193840500EFB0DFA993072000FC
:104C40008326C405232EF40483278405130710004C
:104C50001309050093871700232CF4046396E608D4
:104C60008327840263860700737004306F0000009E
:104C700097C701009387478083A70700639A0708B7
:104C80009309440013850900EFB01FB517C7010051
:104C9000130747808327C402032707006376F700C2
:104CA00017B701002328F77E13074001B387E702F7
:104CB00017C501001305C590938509003305F5005C
:104CC000EFB05FA997B701009387477E83A70700DE
:104CD0000327C40283A7C70263F8E70063860400C2
:104CE0009307100023A0F400032481018320C10155
:104CF000832441018329C10013050900032901010F
:104D0000130101026FB09F9C737004306F000000AC
:104D10009305840117C5010013058599EFB09FA382
:104D20006FF05FFA9307050063080506737004309F
:104D300017B701001307C77583260700639E060295
:104D400003A6C70593062000130500006316D600CE
:104D500023AE07041305100083270700638C0700A8
:104D600097B701009387877403A7070003274704B9
:104D7000631C07026780000097B6010093860673E4
:104D800003A6060083A60600832646049386160023
:104D90002322D6046FF0DFFA97B7010093870771DB
:104DA00083A707006FF09FF803A7070083A60700FB
:104DB000832747049387F7FF2322F70483A746043A
:104DC000E39A07FA7360043067800000130101FB67
:104DD00023229104232E3103232C4103232A510340
:104DE000232861032326710323261104232481042D
:104DF0002320210523248103232291032320A103BF
:104E000097B901009389896B17BB0100130B4B6A9B
:104E100097B401009384046A97BA0100938ACA691F
:104E2000130A1000930B900083A7090003A7070043
:104E30006304071883A7C70003A90700EFD09FCF1B
:104E4000EFD0DFD083270B00130C05006366F50E4F
:104E500097B7010023AEA7641306000063742525ED
:104E600003A50400B3058941EFC01FCCEFE00F801C
:104E70006304051803A50400930600001306000050
:104E800093050100EFC08FCAE30005FA83270100F4
:104E90000324810063D00702832741008325C100DA
:104EA00013050400E780070083270100E3C407FC23
:104EB000032481008327440163860700130544000F
:104EC000EFB09F91EFD09FC883270B00130C050014
:104ED0006362F50C8327010017B70100232A875D61
:104EE000E3EAFBF8B317FA0013F707216316072E5E
:104EF00013F7770C6316072693F70702E38C07F680
:104F000013050400EF00D05C6FF0DFF683A7C70045
:104F100003A4C70083AC070013094400130509006C
:104F2000EFB09F8B8327440213050400E78007003E
:104F30008327C4016386470D83A7090003A70700E1
:104F4000E31607FC03A70A0097B6010023A28657C1
:104F500097B6010023A2F65697B7010023A0E756A3
:104F6000EFD0DFF06FF01FF183A7C70003A9C700E0
:104F700003AD0700930C490013850C00EFB0DF85EB
:104F80008327490213050900E78007008327C90129
:104F9000638C470B83A7090003A70700E31607FCF0
:104FA00003A70A0097B6010023A8F65097B701009F
:104FB00023A6E7506FF01FF2EFD0DFB7EFD01FB995
:104FC00083270B00130C0500E368F5F683A70A009E
:104FD00003A504001309000003A60700B3058941D7
:104FE00017B701002326874D13361600EFC0DFB335
:104FF000EFD0DFE7E31005E8EFB08FD96FF09FE760
:105000008327840193050900B387FC0063E2FC0851
:1050100083A704006386070223280100232A910145
:10502000232C8100EFF0CF9B03A504009306000022
:105030001306000093050101EFB0DFAFE31E05EE9C
:10504000737004306F0000008327890193850C0082
:10505000B307FD006362FD0883A7040063860702AF
:1050600023280100232AA101232C2101EFF04F97CF
:1050700003A5040093060000130600009305010138
:10508000EFB05FABE31805F0737004306F00000001
:1050900003A509002322F40023288400EFB08FEE3B
:1050A0006FF09FE9EFD09FDC83A7090083A7C700BB
:1050B00003A4C700930C440013850C00EFB0CFF19C
:1050C0008327C40163844703832744021305040034
:1050D000E78007006FF01FDA03A509002322F9001B
:1050E00023282901EFB00FEA6FF0DFEA832784015C
:1050F000232884003307F9002322E400636AEC04C8
:10510000330C2C41636EFC0283A704006386070204
:1051100023280100232A2101232C8100EFF04F8C4A
:1051200003A5040093060000130600009305010187
:10513000EFB05FA0E31A05F8737004306F00000051
:1051400003A50A0093850C00EFB0CFE36FF0DFF703
:1051500003A5090093850C00EFB0CFE26FF0DFF6F6
:105160008327410083268401232884003387D700C6
:105170002322E400636AEC0AB307FC4063EED7081D
:105180008327440213050400E78007008327C40136
:10519000E39247CF832684018327410003A70400BD
:1051A000B387D7006306070223280100232AF100F2
:1051B000232C8100EFF0CF8203A5040093060000AA
:1051C0001306000093050101EFB0DF96E31405CA52
:1051D000737004306F00000083274100232CF4001B
:1051E00063880702B38787012322F4002328840001
:1051F000930544006368FC0003A50A00EFB08FD854
:105200006FF05FC703A50900EFB0CFD76FF09FC65F
:10521000737004306F00000003A50A00930544007A
:10522000EFB04FD66FF01FC56374FC00E37AF7F45C
:1052300003A5090093054400EFB0CFD46FF09FC3DE
:10524000130101FF23248100232611002322910052
:105250002320210117B401001304C425EFF00F9897
:105260008327040063840704EFF08F9A83270400E8
:10527000638A0702930800001308000093070000E8
:1052800013072000930600001306004097B50100A5
:105290009385C51217050000130585B3EFC01F9D48
:1052A00063140506737004306F00000017B9010025
:1052B0001309C94313050900EFB04FC797B40100A4
:1052C0009384044413850400EFB04FC61306000016
:1052D000930500011305400097B7010023A0271F85
:1052E00097B7010023AA971CEFB0CFF017B70100C2
:1052F0002322A71C6306050297B501009385850B41
:10530000EFC04FEF6FF05FF68320C10003248100F0
:10531000832441000329010013010101678000007B
:10532000737004306F000000638A050A130101FDE9
:10533000232A5101930A05001305C0022324810288
:105340002322910223202103232E3101232C41010A
:105350002326110223286101232671011309070066
:1053600093890600130A060093840500EF00407E2F
:1053700013040500630C0502EFF04F8697B7010098
:105380009387471383A70700638E0704EFF04F88C6
:105390001305440023205401232C9400232E4401A0
:1053A0002320340323222403EFB04FBA1305040053
:1053B0008320C102032481028324410203290102C4
:1053C0008329C101032A8101832A4101032B0101A1
:1053D000832BC10013010103678000007370043048
:1053E0006F00000097BB0100938B4B3013850B00BF
:1053F000EFB0CFB317BB0100130B8B3013050B00BD
:10540000EFB0CFB213060000930500011305400072
:1054100097B7010023A4770B97B7010023AE670964
:10542000EFB04FDD17B701002326A708630A050078
:1054300097B50100938505F8EFC0CFDB6FF01FF53E
:10544000737004306F000000630E0506130101FE47
:10545000232C8100232E1100232A910017B4010070
:1054600013044405832804001308050013050000F5
:1054700063800804930407002320B100138706000B
:105480002322C100232401019306500063C0B60407
:10549000EFE01FD593072000630EF50403250400F9
:1054A000930600001306000093050100EFB08FE89B
:1054B0008320C101032481018324410113010102DE
:1054C00067800000737004306F00000093050100D6
:1054D000930600001306070013850800EFB05FB7BE
:1054E0008320C101032481018324410113010102AE
:1054F0006780000003250400930600001386040063
:1055000093050100EFB00FE36FF09FFA630605000B
:105510000325050067800000737004306F000000F1
:1055200063160500737004306F000000130101FF63
:10553000232611002324810013040500EFE01FEA55
:10554000032544013334A000EFE09FEC1305040071
:105550008320C10003248100130101016780000042
:1055600063160500737004306F000000130101FF23
:10557000232481001304050023261100EFE01FE619
:1055800003240402EFE0DFE88320C10013050400D8
:1055900003248100130101016780000063160500E8
:1055A000737004306F000000130101FF2324810099
:1055B0002322910013840500930405002326110083
:1055C000EFE0DFE123A08402032481008320C100F7
:1055D00083244100130101016FE09FE3130101FEE9
:1055E000232E110097B701009387C7EC2322A10057
:1055F00003A50700938706002324B1002326C100DA
:105600009305010013860700930600009307E0FF4F
:105610002320F100EFB0DFA38320C10113010102B9
:105620006780000097B701009387C7E883A8070049
:1056300063960800737004306F000000130101FED0
:10564000930706001387050013080500138606005C
:105650009305010013850800930600009308F0FFEE
:10566000232E110023201101232201012324E10014
:105670002326F100EFB00FCC8320C10113010102FA
:1056800067800000630C0500B70700FFB3F7F50063
:10569000638A0700737004306F0000007370043079
:1056A0006F000000130101FF2324810023229100D9
:1056B000232611001304050093840500EFE01FD298
:1056C0000327040093C7F4FFB377F7002320F40007
:1056D000032481008320C1008324410013010101C0
:1056E0006FE01FD3630C0500370700FFB3F7E50039
:1056F000638A0700737004306F0000007370043019
:105700006F0000006F300033130101FF1305C0016B
:105710002324810023261100EF0080431304050099
:10572000630805002320050013054500EFB00F8036
:10573000130504008320C10003248100130101012B
:105740006780000063020502B70700FFB3F7F500AA
:1057500063860700737004306F000000639A0500D1
:10576000737004306F000000737004306F0000002D
:10577000130101FE232C810023282101232631015E
:105780002324410123225101232E1100232A9100B9
:105790009309070013890600930A06001384050085
:1057A000130A0500EFE0DFA3631805006386090014
:1057B000737004306F000000EFD0CFB783240A006D
:1057C000B3779400631209046382070463880A00B4
:1057D0009347F4FFB3F797002320FA00EFD00FE9C7
:1057E0008320C101032481011385040003290101E1
:1057F000832441018329C100032A8100832A4100B7
:105800001301010267800000E302F4FCE38809FC55
:10581000B33550019395850163060900B70700046D
:10582000B3E5F50013860900B3E5850013054A00CA
:10583000EFE04FCDEFD08FE363140500EFA05FD50D
:10584000EFE09FC1931765009309050063DA070035
:10585000B70400019384F4FFB3F499006FF05FF88C
:10586000EFE0DFB783290A00B37734016310090240
:10587000638A070063880A009347F4FFB3F7370190
:105880002320FA00EFE0DFB86FF09FFCE31CF4FE8A
:105890006FF05FFE630C0500B70700FFB3F7F5007C
:1058A000638A0700737004306F0000007370043067
:1058B0006F000000130101FF232481001304050081
:1058C00023261100232291002320210113890500A2
:1058D000EFE0DFB0832404009345F9FFB3F79500B0
:1058E0002320F400EFE0DFB28320C1000324810015
:1058F00013850400032901008324410013010101E1
:1059000067800000138605009306000093050500DC
:1059100017050000130545D76FF05FCC130101FF99
:10592000232481001304050023261100EFA09FDA31
:1059300003240400EFA09FD98320C10013050400B5
:10594000032481001301010167800000630C05003E
:10595000370700FFB3F7E500638A07007370043070
:105960006F000000737004306F0000006F30800C17
:10597000B70700FFB377F600638607007370043043
:105980006F00000063160600737004306F000000A3
:10599000130101FE232C810023282101232631013C
:1059A00023244101232E1100232A9100138906008C
:1059B00093890500130A050013040600EFE05F82D7
:1059C000631E050463060900737004306F00000055
:1059D000EFD04F9683240A009385090013050A002F
:1059E000B3E49900EFF09FF6B3779400630AF408EC
:1059F00083240A00EFD08FC78320C10103248101D3
:105A00001385040003290101832441018329C10076
:105A1000032A81001301010267800000EFD08F91FB
:105A200083240A009385090013050A00B3E43401B6
:105A3000EFF0DFF1B3F7840063848704E30A09FA27
:105A4000B705000513060900B365B40013054A0045
:105A5000EFE04FABEFD08FC163140500EFA05FB351
:105A6000EFE09F9F931765009304050063D407023E
:105A7000B70700019387F7FFB3F4F4006FF0DFF787
:105A800083270A001344F4FFB3F787002320FA00AA
:105A90006FF05FF6EFE09F9483240A00B3779400E1
:105AA000639887009347F4FFB3F797002320FA0029
:105AB000EFE01F966FF0DFFB130101FF232481004D
:105AC000232611001304050023229100EFD08F86B6
:105AD0008327440063860702032504019304C4005E
:105AE000631895006F008003032504016308950285
:105AF000B7050002EFE04FCB83274400E39607FE93
:105B000013050400EF00C01C032481008320C100A2
:105B100083244100130101016FD04FB5737004302D
:105B20006F0000009306060013860500930505002C
:105B300017050000130545BB6FF05FAA630605005B
:105B400003258501678000001305000067800000C1
:105B5000130101FF232481002326110013040500F3
:105B6000EFC05FFD97B701009387879583A7070074
:105B7000639C0704B797010017B701001307C7B963
:105B80009387C7FF97B6010023A2E69417B70100D9
:105B9000232CF79217B701002322F7B897B701001B
:105BA0009387479217B701002328F7B69307100091
:105BB00017B70100232E079017B701002324079081
:105BC00017B70100232EF78E63120402EFD00FAA3D
:105BD000EF10C06013040000130504008320C1000F
:105BE0000324810013010101678000001305840074
:105BF000937735006398070CB79701001307F5FFFB
:105C00009387A7FFE3E4E7FC97B601009386068C31
:105C100083A706006F00400103A70700630A07007F
:105C2000938607009307070003A74700E366A7FED4
:105C300017B7010013070789E38AE7F803A70700EE
:105C4000130600011384870023A0E60003A7470082
:105C5000B306A740637ED6023388A7002322D8006C
:105C600023A2A7008325480097B6010093860686E5
:105C70006F0080009306070003A706000326470075
:105C8000E36AB6FE2320E80023A0060103A747002D
:105C900097B701009387C78783A70700B387E740BB
:105CA00017B701002326F786EFD04F9CE30204F2DA
:105CB000130504008320C1000324810013010101A6
:105CC000678000001375C5FF130545006FF0DFF214
:105CD00063080506130101FF232481002326110018
:105CE00013040500EFC01FE5930584FF0326C4FFDE
:105CF00017A701001307877D6F0080001387070037
:105D00008327070083A64700E3EAC6FE232CF4FEA0
:105D10002320B70097A701009387877F03A7070079
:105D20008327C4FF032481008320C100B387E700D9
:105D300017A70100232EF77C130101016FD00F93E9
:105D40006780000097A701009387877C03A5070061
:105D500067800000678000003367B5001377370065
:105D600093070500631207049308D6FFB3081501D3
:105D700013070500938605006378150303A8060042
:105D80001307470093864600232E07FFE36817FF9B
:105D90009347F5FFB387170193F7C7FF9387470032
:105DA000B385F500B307F5003306C50063F4C70CEF
:105DB0009386450013884700B3B6D70033B8050172
:105DC00033E7F50093C61600134818001377370021
:105DD000B3E60601133717003377D700330EF640CA
:105DE00093861700630807061337AE00631407068F
:105DF00013532E0013880500938607001307000035
:105E000083280800130717001308480023A0160171
:105E100093864600E36667FE1377CEFFB385E50001
:105E2000B387E7006306EE0483C6050013871700F7
:105E30002380D700637EC70283C61500138727001F
:105E4000A380D7006376C70203C725002381E7003C
:105E500067800000B307F640B387F500938515000F
:105E600003C7F5FF93861600238FE6FEE398F5FE41
:105E70006780000067800000B367C50093F73700B4
:105E8000B308C5006382070E63761511B307A040FF
:105E900093F73700138737009306500093F5F50FFB
:105EA000130815003383A8401306F6FF6374D70068
:105EB000130750006368E60E6380070E2300B500E9
:105EC00013071000638EE700A300B500130730002E
:105ED000130825006396E700130835002301B50079
:105EE0001396850033E6C500139705013367E60076
:105EF0003303F34093968501B366D700135623000E
:105F0000B307F5001307000023A0D70013071700FD
:105F100093874700E36AC7FE1377C3FFB307E80020
:105F20006300E3082380B70013871700637C17031F
:105F3000A380B70013872700637617032381B70078
:105F40001387370063701703A381B70013874700D7
:105F5000637A17012382B700138757006374170110
:105F6000A382B7006780000093F5F50F13978500B3
:105F7000B365B700139705013367B700E37415FFE6
:105F8000930705009387470023AEE7FEE3EC17FF76
:105F90006780000067800000130805006FF05FF461
:105FA00067800000930705006FF0DFF78347050067
:105FB00013070500638C07001305150083470500D0
:105FC000E39C07FE3305E5406780000013050000F1
:105FD00067800000130515008347F5FF93851500C2
:105FE00003C7F5FF63880700E386E7FE3385E740D4
:105FF00067800000930700006FF05FFF93070500C4
:106000009385150003C7F5FF93871700A38FE7FE5D
:10601000E31807FE6780000083460500930700022F
:106020006398F6001305150083460500E38CF6FE21
:10603000938756FD93F7D70F6380070493070500F6
:10604000930500006388060413050000938717007A
:10605000138606FD1317250083C607003305A70026
:10606000131515003305A600E39206FE63840500B0
:106070003305A04067800000938536FD83461500F8
:1060800093B5150093071500E39006FC1305000077
:106090006FF0DFFD130500006780000083A7050097
:1060A0002380A70083A705009387170023A0F5008E
:1060B0006780000097A601009386C64183A706006B
:1060C000173703001307076813861700B307F70095
:1060D0002380A70097A5010023AEC53E9307A0002B
:1060E000630AF500930700046308F6001305000037
:1060F00067800000E30C06FE370610F01307170058
:106100008347F7FF2320F6F083A706009387F7FF66
:1061100097A5010023A0F53CE39207FE13050000BC
:1061200067800000130101EB232291142320211525
:10613000232A511323248113232611142324811489
:10614000232E3113232C411323286113232671138B
:10615000232291132320A113232EB11193040500B0
:10616000138905002326C100130C5002930A9000E6
:106170008347090063888703638C070603A4040030
:106180006F008000638607062300F40003A4040068
:10619000130919001304140023A084008347090085
:1061A000E39287FF034619009308190093860800BD
:1061B000130D00029309F0FF130AF0FF130800000B
:1061C000130550059307D6FD93F7F70F13891600B3
:1061D000636EF53A17A701001307C7E293972700EC
:1061E000B387E70083A70700B387E700678007004E
:1061F0008320C1140324811483244114032901142E
:106200008329C113032A8113832A4113032B01130A
:10621000832BC112032C8112832C4112032D0112F6
:10622000832DC1111301011567800000930C8000BC
:10623000232401009307100063DA071D8327C100A0
:1062400003A40400938B770093F68BFF03AB060047
:1062500083A94600938786002326F10013860C004D
:106260009306000013050B0093850900EF204030D2
:106270002328A1009307000063803733930D410169
:10628000930B100013860C009306000013050B00FF
:1062900093850900EF10906A9306000013860C00A6
:1062A000130B050093890500EF20802C83278100C4
:1062B00023A0AD0093861B00938D4D0063863701AC
:1062C000938B06006FF01FFCE37C9BFF63D24603B9
:1062D000930704002380A70103A40400130AFAFF14
:1062E0009307140023A0F40013840700E3C446FFBF
:1062F00093962B0093070101B386D7006F008002AD
:10630000938777052300F40003A40400938BFBFF1D
:1063100093871B001304140023A084009386C6FFF8
:10632000E358F0E483A70600E3ECFAFC9387070345
:106330006FF05FFD83A70400930600030327C100ED
:106340002380D70083A7040093064700930C000125
:106350001386170023A0C40013068007A380C7007C
:1063600003A404002324010093070700130414006E
:1063700023A0840003AB0700930900002326D1006B
:106380006FF0DFED8327C10083AC0700938B4700DC
:1063900063880C28635C40259307D002631EFD20B0
:1063A00083C70C006388070263D8092483A604000E
:1063B000938C1C00130AFAFF2380F60003A4040048
:1063C0001304140023A0840083C70C00E39E07FC81
:1063D0006352400303A40400930700022300F40067
:1063E00003A40400130AFAFF1304140023A084007A
:1063F000E3160AFE232671016FF09FD723240100C4
:1064000093071000930CA000E3CA07E38327C100A1
:1064100003A40400938647006FF0DFF503C616005F
:10642000930609006FF01FDA83A704009306500259
:106430002380D70003A404001304140023A08400C5
:106440006FF01FD3930C0001232401006FF09FDE37
:106450008327C10003C616009306090083A907001D
:10646000938747002326F100E35E0AD4138A0900CC
:106470009309F0FF6FF01FD503C61600130DD0026D
:10648000930609006FF01FD49347FAFF93D7F741A3
:1064900003C61600337AFA00930609006FF09FD204
:1064A00003C61600130D0003930609006FF09FD179
:1064B00083C51600930906FD93060900938705FD21
:1064C00013860500E3E2FAFA93972900B3893701AE
:1064D0009386160093991900B389B90083C5060005
:1064E000938909FD938705FD13860500E3FEFAFCF9
:1064F0006FF09FF70327C10083A7040083260700DE
:10650000130747002326E1002380D70003A40400DB
:106510001304140023A084006FF09FC5930710009C
:1065200063D4070F8327C1009386770093F686FF15
:10653000938786002326F10083A9460083A70600DF
:1065400063DE090E83A604001306D002B307F040F1
:106550002380C60003A40400B336F000B309304121
:106560001304140023A08400138B0700B389D940BF
:10657000930CA000232401006FF05FCE03C6160029
:1065800013081800930609006FF0DFC383A7040007
:10659000138908006FF09FE9E3729BCF9307100007
:1065A000930B000093061000E3C447D36FF05FD451
:1065B00097AC0100938C0CE19385090013850C00C6
:1065C000EF100070330AAA406352400303A4040092
:1065D0002300A40103A40400130AFAFF1304140007
:1065E00023A08400E3160AFE130A000083C70C00F0
:1065F000E38207E0E3CC09DA9389F9FF1307F0FFA0
:10660000E396E9DA6FF0DFDC8327C1009386470069
:1066100083A707002326D10093D9F7416FF05FF2DB
:10662000635640019307D002E314FDF897AC0100D4
:10663000938C4CD9930780026FF01FD7138B070000
:10664000930CA0002324010003A404006FF01FC1D9
:10665000130101EB232E3113B70900409387F9FF93
:106660002324811423229114232C4113232A511310
:1066700023261114232021152328611323267113A7
:1066800023248113232291132320A113232EB1113C
:10669000130A05002324B10017A40100130484E3A6
:1066A000973A0300938A0A0A97A40100938404ABE3
:1066B0002326F100930550021305A00013080004DF
:1066C000B70610F083470A00638EB7046388070A91
:1066D00003270400130A1A00130617003387EA0081
:1066E00097A8010023A8C8DE2300F7006380A7084D
:1066F000E31A06FD173703001307C7041307170033
:106700008347F7FF23A0F6F0832704009387F7FF62
:1067100017A601002320F6DCE39207FE83470A0058
:10672000E396B7FA83461A0013051A00130705000B
:10673000930B0002130BF0FF130CF0FF1308000083
:1067400093055005930890009387D6FD93F7F70FB4
:10675000130A170063ECF54493972700B38797005B
:1067600083A70700B38797006780070017370300E8
:10677000130747FDE31406F86FF0DFF48320C1141C
:106780000324811483244114032901148329C11390
:10679000032A8113832A4113032B0113832BC11274
:1067A000032C8112832C4112032D0112832DC11160
:1067B0001301011567800000930C8000130D000089
:1067C0009307100063DA07218327810093877700FE
:1067D00093F787FF83AD070003AB4700138787005C
:1067E0002324E10013860C009306000013850D009E
:1067F00093050B00EF10D0572328A10063086D45C7
:10680000130941019309100013860C009306000040
:1068100013850D0093050B00EF10501213860C002A
:1068200093060000930D0500138B0500EF105054E4
:106830002320A9009389190013094900E3166DFD6F
:10684000E3F49DFD13060004B70610F063D489033A
:106850008327040013871700B387FA0097A5010068
:1068600023AAE5C623807701630AC706130CFCFF41
:10687000E3C089FF8327C1001305C100930890007E
:10688000B386F9009396260093070101B386D700DB
:106890001308A00013030004370610F0E38CA6E0F1
:1068A00083A706009305000363F4F80093057005C1
:1068B00003270400B387B700930517003387EA0066
:1068C00017AE01002328BEC02300F70063860737F8
:1068D000638C65329386C6FF6FF05FFC1737030049
:1068E000130747E6130717008347F7FF23A0F6F0C7
:1068F000832704009387F7FF97A5010023ACF5BC1D
:10690000E39207FE130CFCFF6FF09FF68327040051
:10691000130600041387170097A5010023ACE5BAFE
:10692000B386FA00930500032380B6006308C750BE
:106930009387270097A6010023AEF6B83387EA00B5
:10694000930680072300D70017370300130787DF5C
:10695000B70610F06392C702130717008347F7FFCB
:1069600023A0F6F0832704009387F7FF17A6010002
:106970002322F6B6E39207FE83278100930C0001E1
:10698000130D00009387470003278100130B0000BD
:10699000832D07002324F1006FF0DFE483278100BB
:1069A00083AC070013894700638E0C4C6358802B1F
:1069B0009307D0026394FB3E03C70C0093050700C6
:1069C0006314072A6F00002F93071000930CA00098
:1069D000130D0000E3CA07DF832781009387470078
:1069E0006FF09FFA832781008346170013070A0080
:1069F00003AB0700938747002324F100E3560CD430
:106A0000130C0B00130BF0FF6FF01FD4834617001D
:106A1000930BD00213070A006FF01FD39347FCFFBC
:106A200093D7F74183461700337CFC0013070A0015
:106A30006FF09FD183461700930B000313070A00E2
:106A40006FF09FD003461700138B06FD13070A0053
:106A5000930706FD93060600E3E2F8FA93172B006E
:106A6000B38767011307170093971700B387C70011
:106A700003460700138B07FD930706FD93060600E8
:106A8000E3FEF8FC6FF09FF7832581008327040065
:106A90001306A00003A7050093861700B387FA002A
:106AA00017A501002328D5A22380E70013894500FC
:106AB0006300C736930700046384F62A2324210168
:106AC0006FF05FBF9307100063DE073583278100F7
:106AD00013877700137787FF930787002324F1003C
:106AE000032B47008327070063560B3E0327040050
:106AF000130600049306170097A5010023ACD59C4C
:106B00003387EA009305D0022300B700638CC638B0
:106B1000B307F0403337F000330B6041938D07002B
:106B2000330BEB40930CA000130D00006FF09FCBD4
:106B3000834617001308180013070A006FF0DFC020
:106B40008346170013070A006FF01FC08327040055
:106B5000930600041387170017A60100232CE6965E
:106B6000B387FA00130650022380C700E314D7B49A
:106B700017370300130707BDB70610F013071700F8
:106B80008347F7FF23A0F6F0832704009387F7FFDE
:106B900017A601002320F694E39207FE6FF09FB141
:106BA000930C0001130D00006FF09FC183270400B8
:106BB00093060004130A05001387170017A60100A7
:106BC000232AE690B387FA00130650022380C700F9
:106BD000E312D7AE173703001307C7B6B70610F096
:106BE000130717008347F7FF23A0F6F0832704005D
:106BF0009387F7FF17A60100232EF68CE39207FE7A
:106C0000130A05006FF01FAB17370300130787B394
:106C1000130717008347F7FF2320F6F083270400AC
:106C20009387F7FF97A5010023A6F58AE39207FE55
:106C30009386C6FF6FF09FC617370300130787B010
:106C4000E39805FC9386C6FF6FF05FC5E3FA9DBB32
:106C5000930910006FF01FBF130C000003C70C0056
:106C600093050700E30C07E49308F0FF1305A00069
:106C700013080004B70610F0635E0B0C83270400B2
:106C800013861700B387FA0017A301002324C384D7
:106C90002380E7006382A5086308060B938C1C0021
:106CA00003C70C00130CFCFF93050700E31607FC59
:106CB000E35680E1832704009305000213060004D5
:106CC000B70610F06F00C000130CFCFFE3080CDEE9
:106CD00013871700B387FA002380B70017950100C8
:106CE000232AE57E93070700E310C7FE173703004A
:106CF000130747A5130717008347F7FF23A0F6F0F4
:106D0000832704009387F7FF179501002324F57C60
:106D1000E39207FE6FF05FFB17370300130787A2AC
:106D2000E30E06F6130717008347F7FF23A0F6F0DC
:106D3000832704009387F7FF17960100232CF6782A
:106D4000E39207FE6FF09FF5173703001307879F45
:106D50006FF05FFD130BFBFFE3121BF36FF05FF5AA
:106D6000173703001307079EB70610F01307170025
:106D70008347F7FF23A0F6F0832704009387F7FFEC
:106D8000179601002328F674E39207FE23242101BD
:106D90006FF05F92979C0100938CCC6293050B007F
:106DA00013850C00EF00D071330CAC40E35880EB3E
:106DB0008327040013060004B70610F06F00C0001C
:106DC000130CFCFFE30A0CE813871700B387FA00E3
:106DD000238077019795010023AEE56E93070700A6
:106DE000E310C7FE173703001307C79513071700F3
:106DF0008347F7FF23A0F6F0832704009387F7FF6C
:106E00009795010023A8F56CE39207FE6FF05FFBF6
:106E10001737030013070793E39806F4232421018F
:106E20006FF05F89832781001387470083A70700DE
:106E30002324E10013DBF7416FF01FCB173703006A
:106E400013074790B70610F0130717008347F7FFA3
:106E500023A0F6F0832704009387F7FF179601001D
:106E6000232AF666E39207FE9307100017970100A6
:106E70002322F76693078007173703002304F78C54
:106E80006FF09FAF635680019307D002E394FBF04D
:106E9000979C0100938C0C5313078002930580028A
:106EA0006FF09FDC973603009386C689370610F093
:106EB0009386160003C7F6FF2320E6F0032704009D
:106EC0001307F7FF9795010023A6E560E31207FE7D
:106ED0006FF01FC4938D0700930CA000130D0000EA
:106EE0006FF05F90B70710F023A0A7F26F000000CB
:106EF000130101FC130341022322B1029305030095
:106F0000232E11002324C1022326D1022328E102CB
:106F1000232AF102232C0103232E110323266100CF
:106F2000EFF00FF38320C1011305000013010104EA
:106F300067800000130101FB1303810323248102F6
:106F40002326A100232CC10213040500130603000D
:106F50001305C100232611022322F104232ED1029E
:106F60002320E1042324010523261105232E61009B
:106F7000EFF04F9B8327C100238007000325C1004A
:106F80008320C102330585400324810213010105DA
:106F900067800000B70710F083A647F403A607F444
:106FA00003A747F4E31AD7FEB7160000938606FA44
:106FB000B306D60033B6C600B305E60023A4D7F463
:106FC00023A6B7F467800000B70710F003A747F4C3
:106FD00003A607F483A647F4E31AD7FEB71600000A
:106FE000938606FAB306D60033B6C60023A4D7F4B8
:106FF000B305E60023A6B7F49307000873A0473053
:1070000067800000130101FF232481002326110063
:10701000130440011304F4FFEF00502FE31C04FE9F
:107020008320C10003248100130101016780000057
:10703000130101FF232481002326110097970100EB
:107040009387C749179401001304044903A7070055
:10705000832704001306F07C9306470693874706B0
:107060009795010023ACD5469795010023A6F546D8
:10707000634AD6008320C10003248100130101016B
:1070800067800000130747899797010023A8E7440A
:10709000EF00103A930710006316F502032704006F
:1070A000B71700009387F77613050000E3D4E7FCD9
:1070B000EFF05FE3032481008320C100130101018D
:1070C0006FB05FA61795010013054530EFF05FE242
:1070D00013052000EFF01FE1032481008320C1008D
:1070E000130101016FB01FA4179501001305852F2F
:1070F0006FF01FE0179501001305452F6FF05FDF5C
:10710000130101FF23248100232291002326110073
:10711000B7140000179401001304C42D938784381A
:10712000130000009387F7FFE39C07FE130504009C
:10713000EFF01FDC6FF09FFE130101FF232611000B
:1071400023248100EF00D00C170700001307C7EBC2
:107150009306000013061000930520031795010005
:107160001305C529EFE04F9C13040500EFB01F9EE7
:107170001306050013050400032481008320C100C9
:10718000130700009306000093051000130101018E
:107190006FE08FAB130101FF23261100EF00502990
:1071A0001307100093070000631AE5008320C10055
:1071B0001385070013010101678000001795010086
:1071C0001305C520EFF0DFD28320C1009307200014
:1071D00013850700130101016780000073700430FC
:1071E0006F00000067800000737004306F000000C3
:1071F000130101FF232291002320210123261100E6
:107200002324810013090500EFC09FFC979701001C
:107210009387872E83A70700930450006382A70AF1
:10722000179401001304C42D13050000EFC04FFA9A
:10723000032504001307F0FF930600001306100057
:1072400093850400EFE00FD0E31005FE6F0000040B
:10725000EFC00FF8032504009306F0FF1306F000BB
:1072600093050900EFE0CFF01375F5001307F0FF69
:1072700093061000130600009305F000631A9504AE
:1072800003250400EFE00FCC631005041305000094
:10729000EFC00FF4032504009306F0FF1306F0007F
:1072A00093050900EFE0CFEC9374F5009307F0002D
:1072B00013050000E38EF4F8737004306F000000D3
:1072C000930430006FF0DFF5737004306F0000003E
:1072D000737004306F000000130101FE232C810045
:1072E0002326310123244101232E1100232A91005A
:1072F0002328210117940100130484209799010089
:1073000093898920130AF00F13050000EFC04FEC9A
:10731000032504001307F0FF930610001306100066
:1073200093052000EFE00FC21309050003250400B8
:107330001307F0FF93061000130600009305200AC0
:10734000EFE04FC01375250A9307200A930410003D
:107350006308F51213050000EFC08FE70325040052
:107360001307F0FF93061000130610009305200A80
:10737000EFE04FBD630445019304100013050000C6
:10738000EFC00FE5032504009306F0FF1306F0009D
:1073900093052000EFE0CFDD1375F5009307F000B3
:1073A0006304F50093041000032504009305000016
:1073B000EFE0CFD96302050A03250400930500001E
:1073C00093041000EFE00FCD13050000EFC04FE075
:1073D000032504009306F0FF1306F0009305200038
:1073E000EFE00FD91375F5009307F0006304F50083
:1073F000930410000325040093050000EFE00FD56F
:1074000063020502032504001307F0FF9306100032
:10741000130600009305F000EFE0CFB27370043064
:107420006F000000032504001307F0FF930610000F
:10743000130600009305F000EFE0CFB0E31005FE67
:10744000E39E04FC83A709009387170017970100A8
:10745000232CF70A6FF05FEB03250400930500006F
:10746000EFE04FC3631405026392040283A709008F
:1074700093871700179701002328F7086FF0DFF4B0
:107480009304E9F5B33490006FF0DFEC930410003F
:107490006FF09FF3130101FD232021032326110226
:1074A0002324810223229102232E3101232C410126
:1074B000232A5101232861012326710123248101FC
:1074C000232291012320A10113090500EFE0CFA39E
:1074D0009797010023A6A70263020552179A01009D
:1074E000130A8A0103250A009799010093898900EC
:1074F00013041000EFA0DFD79304050003A50900D3
:10750000EFA01FD793073000630EF54E930B80005A
:10751000930A100097940100938484FE130B2000BB
:10752000130C300003250A00EFB04F8B03A50900B0
:10753000EFB0CF8A03250A00EFA09FD36304650153
:107540001304100003A50900EFA09FD26304650196
:107550001304100003A5040093850A00EFE00FBF99
:1075600093F73A0003250A0063980744EFA05FD021
:10757000630465011304100093F75A0003A5090082
:1075800063960742EFA0DFCE630465011304100089
:10759000938BFBFF939A1A00E3960BF803250A00DE
:1075A000179D0100130D8DF6930A2000EFB00F8395
:1075B00003A50900930B1000930C000AEFB00F8293
:1075C00003A50400130B3000130CD005EFE0CFCE61
:1075D000EFE08F939797010023A4A7F2630C054077
:1075E00013050900EFA09FFF13050900EFA05FC876
:1075F000630455011304100003A504009305200A39
:10760000EFE0CFB403A504001307000093060000C9
:10761000130600009305F00FEFE0CF92630495018D
:107620001304100013050900EFA09FC46304550163
:107630001304100003A504009305D00FEFE00FB171
:1076400003A50400130700009306000013060000C2
:107650009305F00FEFE00F8F9307D00F6304F50051
:107660001304100013050900EFA09FC06304550127
:107670001304100003A5040093052000EFE00FADF4
:1076800013050900EFA0DFBE6304650113041000B9
:1076900003A5040093050000EFE04FAB9307F00F44
:1076A0006304F5001304100003A5040093052000F3
:1076B000EFE04F9E9307F00F6304F50013041000F2
:1076C00013050900EFA09FF113050900EFA05FBAB1
:1076D000630455011304100003A504009305200062
:1076E000EFE0CFA613050900EFA09FB86304650182
:1076F0001304100003A50400130700009306000004
:10770000130600009305F00FEFE0CF8363048501BB
:107710001304100003A504009305F00FEFE08F970A
:10772000630485011304100003A504009305000001
:10773000EFE04F96630405001304100013050900E1
:10774000EFA01FB3630465011304100003250A00B2
:10775000EFA01FB2630465011304100003A5090024
:10776000EFA01FB1630465011304100003A504001A
:107770009305E000EFE08F9D03A504009306F0FF62
:107780001306100093051000EFE08F9E137515008F
:10779000631405001304100003A504009305000002
:1077A000EFE04F8F9307E0006304F500130410002F
:1077B00003A504009305E000EFE0CF8D03A50400CE
:1077C00093050000EFE00F8D630405001304100023
:1077D00013050900EFA09FE003250A00EFA01FE0BA
:1077E00003A50900EFA09FDF13050900EFA05FA824
:1077F000630455011304100003250A00EFA05FA7DE
:10780000630455011304100003A50900EFA05FA64F
:10781000630455011304100003A504009306F0FF50
:107820001306F00093051000EFE08F941375F50038
:107830009307F0006304F5001304100003A504008F
:1078400093050000EFE00F856304050013041000AA
:1078500013050900EFA0DFA1630465011304100004
:1078600003250A00EFA0DFA06304650113041000E4
:1078700003A50900EFA0DF9F630465011304100056
:1078800013050900EFA09FD503250A00EFA01FD51F
:1078900003A50900EFA09FD413050900EFA05F9D89
:1078A000630455011304100003250A00EFA05F9C38
:1078B000630455011304100003A50900EFA05F9BAA
:1078C0006304550113041000930520001305000004
:1078D000EFA09FB603A504009306F0FF1306F00087
:1078E00093051000EFE0CF881375F5009307F000C3
:1078F0006304F5001304100003A5040093050000C1
:10790000EFD05FF9630405001304100013050900AC
:10791000EFA01F96630475011304100003250A00ED
:10792000EFA01F95630475011304100003A509005F
:10793000EFA01F94630475011304100013050000E9
:1079400093050000EFA05FAF13050900EFA05F9261
:10795000630455011304100003250A00EFA05F9192
:10796000630455011304100003A50900EFA05F9004
:10797000630455011304100003A50400EFE0CF9346
:1079800013050900EFA0DF8E6304650113041000E6
:1079900003250A00EFA0DF8D6306650303A5090038
:1079A000EFA01F8D737004306F000000EFA05F8C9C
:1079B000E31E85BD6FF0DFBDEFA09F8BE31C85BB91
:1079C0006FF09FBB03A50900EFA09F8AE31C65FD34
:1079D000E31A04FC83270D00938717001797010013
:1079E0002326F7B2EFD05FD29797010023AAA7B062
:1079F000E31805BE737004306F000000737004302C
:107A00006F0000001384D4FF333480006FF01FB088
:107A1000130101FE93080000130800009307C10042
:107A2000130710009306000013060040979501000D
:107A30009385059E170500001305458A232E110026
:107A4000EFA0CFA28326C100930800001308000016
:107A500093070000130700001306004097950100EC
:107A60009385859B17050000130505A3EFA00FA0C4
:107A70009308000013080000979701009387C7A799
:107A8000130710009306400013060040979501006D
:107A90009385059917F5FFFF1305C575EFA00F9D99
:107AA00097970100938707A593080000130800002B
:107AB00013071000930680001306004097950100FD
:107AC0009385059617F5FFFF1305C572EFA00F9A72
:107AD00097970100938707A283A707006380070297
:107AE000EFD09FC29797010023AAA7A0630C0500BF
:107AF0008320C1011301010267800000737004300C
:107B00006F000000737004306F000000130101FF6C
:107B10002326110023248100979701009387479D16
:107B200083A7070013074006938717009796010065
:107B300023A0F69C6382E7021307800C638CE7089E
:107B40001307C0126382E7048320C100032481006D
:107B50001301010167800000179401001304049AC7
:107B600003250400EFD09FDB630805049307100092
:107B700017970100232CF7968320C100032481006E
:107B80001301010167800000979701009387079711
:107B900003A5070093052001EFD0DFD6930710005F
:107BA000630EF504179701002322F79497970100BD
:107BB00023A007946FF05FF903250400130600006B
:107BC00093052001EFD01FF693071000E310F5FA9C
:107BD0006FF09FF7979701009387479203A50700DF
:107BE000EFD0DFD393072001E300F5F693071000F1
:107BF00017970100232CF78E6FF01FF8979701005D
:107C00009387C78E83A70700179701002322078E4B
:107C1000E39C07F2979701009387C78E83A707001D
:107C20009387170017970100232EF78C6FF0DFF171
:107C3000179701001307878D832807009797010086
:107C40009387878C83250700179601001306868982
:107C500083A6070003260600179801001308C888AA
:107C600003270800179501002320B588130500009D
:107C70006306D600330717413335E00003A607003B
:107C80001797010013070788979701009387478587
:107C90008326070083A707000327070097950100A5
:107CA00023A2C584B387D740B337F000B307F040B1
:107CB0009796010023A6E6823375F50067800000E1
:107CC000B305B500930705006386B70003C7070037
:107CD000631607003385A74067800000938717006D
:107CE0006FF09FFE9308000063DC05003305A040A1
:107CF000B337A000B305B040B385F5409308F0FF5B
:107D000063DA06003306C040B337C000B306D04084
:107D1000B386F64013080600138306009307050098
:107D2000138705006398062497860100938686587A
:107D300063F8C50E370E0100637AC60D130EF00FFF
:107D40006374CE0013038000335E6600B386C60101
:107D500003CE0600330E6E00130300023303C3414B
:107D6000630C0300B3956500335EC50133186600EC
:107D70003367BE00B3176500135E0801B355C70330
:107D8000131508011355050193D607013376C70370
:107D9000B305B50213160601B366D60063FAB60042
:107DA000B386060163E6060163F4B600B3860601F6
:107DB000B386B64033F7C6039397070193D70701FD
:107DC000B3D6C603B306D50213150701B367F50092
:107DD00063FAD700B387070163E6070163F4D700AE
:107DE000B3870701B387D74033D5670093050000F9
:107DF000638C0800B307A0403337F000B305B040F0
:107E000013850700B385E54067800000370E000149
:107E100013030001E36AC6F3130380016FF0DFF27E
:107E20006316060013081000335868023707010074
:107E30006372E80A1307F00F6374070113038000ED
:107E400033576800B386E60003C6060033066600B3
:107E5000130300023303C34063180308B3850541CD
:107E600093560801131508011355050113D6070190
:107E700033F7D502B3D5D502131707013367C7000F
:107E8000B305B502637AB7003307070163660701DC
:107E90006374B70033070701B305B74033F7D50262
:107EA0009397070193D70701B3D5D502B305B50260
:107EB00013150701B367F50063FAB700B38707012D
:107EC00063E6070163F4B700B3870701B387B740E0
:107ED0006FF09FF13707000113030001E362E8F63A
:107EE000130380016FF0DFF53318680033DEC5003F
:107EF000935E08013356C500B31765003355DE03A2
:107F0000B39565003366B6009315080193D5050156
:107F1000935606013377DE033385A5021317070155
:107F20003367D700637AA700330707016366070149
:107F30006374A70033070701B306A74033F7D603DE
:107F40001316060113560601B3D6D60313170701FD
:107F5000B386D502B365C70063FAD500B3850501C2
:107F600063E6050163F4D500B3850501B385D5400B
:107F70006FF01FEFE3EED5E63708010063FC06055E
:107F8000930EF00F33B8DE001318380033DE06010D
:107F900017830100130303323303C301834E03002D
:107FA000130E0002B38E0E01330EDE41631E0E026D
:107FB00063E4B600636AC500B307C540B385D54026
:107FC0003335F5003387A540138507009305070077
:107FD0006FF01FE23703000113080001E3E866FABF
:107FE000130880016FF09FFA3357D601B396C6018C
:107FF000B366D700B357D50133D7D501B395C501C3
:10800000B3E7B70093D506013373B702139F060198
:10801000135F0F0113D807013316C6013315C501CD
:108020003357B7021313030133680301B30FEF0291
:1080300013030700637EF8013308D8001303F7FF2A
:108040006368D8006376F8011303E7FF3308D800AC
:108050003308F841B37FB8023358B802939F0F0139
:10806000B3050F03139F0701135F0F0133EFEF01F8
:1080700013070800637EBF00330FDF001307F8FF0C
:108080006368DF006376BF001307E8FF330FDF008C
:1080900013130301B70F01003363E3009387FFFF5E
:1080A00013580601330FBF40B375F3001353030198
:1080B000B377F6003387F502B307F302B385050300
:1080C00033030303B385F500135807013308B800E1
:1080D0006374F8003303F301B70701009387F7FFD8
:1080E000935508013378F800131808013377F70027
:1080F000B38565003307E8006366BF00631EBF00F9
:10810000637CE5003306C7403337C700B385D540ED
:10811000B385E540130706003307E5403335E50036
:10812000B305BF40B385A540B397D5013357C70109
:1081300033E5E700B3D5C5016FF09FCB938705000A
:10814000130806001387060013030500639606282C
:10815000978801009388081663F6C50E370701005B
:108160006378E60C1307F00F3337C7001317370097
:10817000B356E600B388D80083C608003387E6000C
:1081800093060002B386E640638C0600B397D700DF
:108190003357E5003318D600B365F7003313D50025
:1081A00013550801B3D7A50213160801135606018B
:1081B0009356030133F7A502B305F602131707011F
:1081C000B366D7001387070063FEB600B3860601C7
:1081D0001387F7FF63E8060163F6B6001387E7FF2E
:1081E000B3860601B386B640B3F7A60213130301A4
:1081F00013530301B3D6A6029397070133E3670035
:10820000B305D60213850600637CB3003303680010
:108210001385F6FF636603016374B3001385E6FFFD
:10822000131707013367A700930500006F00400E86
:10823000B706000113070001E36CD6F213078001B3
:108240006FF01FF3631606009306100033D8C602C2
:10825000B70601006372D80C9306F00F63F40601B1
:1082600013078000B356E800B388D80083C608001F
:10827000B386E600130700023307D7406318070AE6
:10828000B38707419305100013560801931808019E
:1082900093D808019356030133F7C702B3D7C70237
:1082A00013170701B366D7003385F8021387070059
:1082B00063FEA600B38606011387F7FF63E8060195
:1082C00063F6A6001387E7FFB3860601B386A640D0
:1082D000B3F7C6021313030113530301B3D6C60247
:1082E0009397070133E36700B388D802138506002C
:1082F000637C1301330368001385F6FF6366030193
:10830000637413011385E6FF131707013367A70092
:108310001305070067800000B7060001130700017E
:10832000E362D8F4130780016FF0DFF33318E8003D
:10833000B3D5D7003313E500B356D5001355080164
:10834000B397E70033F7A502B3E8F60093170801E7
:1083500093D7070113D60801B3D5A5021317070158
:108360003367C700B386B70213860500637ED70064
:10837000330707011386F5FF636807016376D700AB
:108380001386E5FF33070701B306D74033F7A6028C
:108390009398080193D80801B3D6A60213170701D2
:1083A000B385D702B36717011387060063FEB700D2
:1083B000B38707011387F6FF63E8070163F6B70089
:1083C0001387E6FFB3870701B387B740931506010C
:1083D000B3E5E5006FF05FEB63E6D5183707010002
:1083E00063F4E6041308F00F3337D800131737008F
:1083F00033D8E600978501009385C5EBB385050169
:1084000003C80500930500023308E800B385054161
:108410006396050213071000E3ECF6EE3335C50052
:10842000134715006FF0DFEEB705000113070001D9
:10843000E3E0B6FC130780016FF09FFB33570601A2
:10844000B396B600B366D70093DE060133D70701B3
:10845000B378D703B397B700335805013363F800F7
:108460009397060193D70701135803013316B600FB
:108470003357D7039398080133E80801338FE70295
:10848000130E0700637EE8013308D800130EF7FFD0
:108490006368D8006376E801130EE7FF3308D8005D
:1084A0003308E841B378D8033358D80393980801C8
:1084B000B38E07039317030193D70701B3E7F800BF
:1084C0001307080063FED701B387D7001307F8FF2F
:1084D00063E8D70063F6D7011307E8FFB387D70037
:1084E000131E0E01B387D741B70E01003367EE00AC
:1084F0001388FEFF33730701935807013378060191
:1085000013560601330E03033388080393560E01F6
:108510003303C30233030301B3866600B388C80282
:1085200063F40601B388D80113D60601B308160117
:1085300063E61703E39A17CFB70701009387F7FFA6
:10854000B3F6F60093960601337EFE003315B500B0
:10855000B386C60193050000E37CD5DA1307F7FF65
:108560006FF09FCC93050000130700006FF05FDAF7
:10857000930806001387060093070500138805007B
:10858000639C0622978601009386C6D263FCC50CC5
:1085900037030100637E660A1303F00F6374C300A0
:1085A000130780003353E600B386660003CE06004F
:1085B00013030002330EEE003303C341630C0300C8
:1085C000B3956500335EC501B31866003368BE001D
:1085D000B317650013D608013377C8021395080155
:1085E0001355050193D607013358C8021317070125
:1085F000B366D7003308050363FA0601B386160194
:1086000063E6160163F40601B3861601B3860641DC
:1086100033F7C6029397070193D70701B3D6C60273
:10862000B306D50213150701B367F50063FAD70047
:10863000B387170163E6170163F4D700B387170107
:10864000B387D74033D567009305000067800000EB
:108650003703000113070001E36666F41307800186
:108660006FF05FF46316060013061000B35816038C
:108670003706010063F2C80A1306F00F637416018F
:108680001307800033D6E800B386C60003CE060089
:1086900013030002330EEE003303C34163180308D3
:1086A000B385154113D7080113950801135505012A
:1086B00013D60701B3F6E502B3D5E502939606019A
:1086C000B3E6C600B305B50263FAB600B386160179
:1086D00063E6160163F4B600B3861601B385B640AF
:1086E000B3F6E5029397070193D70701B3D5E502E7
:1086F000B305B50213950601B367F50063FAB70039
:10870000B387170163E6170163F4B700B387170156
:10871000B387B7406FF01FF337060001130700015E
:10872000E3E2C8F6130780016FF0DFF5B398680045
:1087300033D7C501B3176500335EC50113D50801F2
:10874000B376A702B3956500336EBE00939508011A
:1087500093D5050113560E013357A70293960601D0
:10876000B3E6C6003387E50263FAE600B386160176
:1087700063E6160163F4E600B38616013386E6402D
:10878000B376A602131E0E01135E0E013356A60227
:10879000939606013386C502B3E5C60163FAC500A8
:1087A000B385150163E6150163F4C500B3851501B2
:1087B000B385C5406FF01FEFE3EAD5E83707010046
:1087C00063FCE604930EF00F33B7DE001317370097
:1087D00033D3E600978801009388C8ADB38868005A
:1087E00083CE0800130E0002B38EEE00330EDE417E
:1087F000631E0E0263E4B600636AC500B307C5409A
:10880000B385D5403335F5003388A540138507007F
:10881000930508006FF09FE3B708000113070001FC
:10882000E3E816FB130780016FF09FFA3357D60178
:10883000B396C601B366D700B357D50133D7D50178
:10884000B395C501B3E7B70093D506013373B702FB
:10885000139F0601135F0F0193D807013316C6015A
:108860003315C5013357B70213130301B36813015E
:108870003308EF021303070063FE0801B388D80032
:108880001303F7FF63E8D80063F608011303E7FF5B
:10889000B388D800B3880841B3FFB802B3D8B80290
:1088A000939F0F01B3051F03139F0701135F0F0170
:1088B00033EFEF0113870800637EBF00330FDF0043
:1088C0001387F8FF6368DF006376BF001387E8FF54
:1088D000330FDF0013130301B70801003363E30014
:1088E0009387F8FF13580601330FBF40B375F300A9
:1088F00013530301B377F6003387F502B307F3028E
:10890000B385050333030303B385F500135807014B
:108910003308B8006374F80033031301B70701008C
:108920009387F7FF935508013378F800131808016F
:108930003377F700B38565003307E8006366BF004F
:10894000631EBF00637CE5003306C7403337C700B2
:10895000B385D540B385E540130706003307E540EE
:108960003335E500B305BF40B385A540B397D501C6
:108970003357C70133E5E700B3D5C5016FF01FCD0D
:1089800097870100938787B283A6070017870100A6
:10899000130787B00327070023A2A600637EE50024
:1089A00017870100130707B00325070083A50700F9
:1089B000938545006F701FDD130101FF23248100A3
:1089C0002326110017870100130707AE13040500C3
:1089D0000325070083A5070093854500EF709FDA04
:1089E00097870100938787A983A707006376F40020
:1089F0009787010023A487A88320C1000324810056
:108A0000130101016780000097870100938707AA7F
:108A100003A7070083A60700832747049387F7FF70
:108A20002322F70483A7460463940700736004308D
:108A300067800000130101FE232C8100232A91008E
:108A40001304050093840500232821012326310106
:108A50002324410123225101232E1100EFA08F8DE9
:108A60008327040003290401B7090001B3E5970037
:108A7000930AC4002320B400930400009389F9FFF3
:108A8000370A00020327040063822A05032609002F
:108A900013050900B3654701B376360193175600F5
:108AA00033F7E6000329490063C607006316070091
:108AB0006FF05FFDE398E6FC9317760063D4070040
:108AC000B3E4D400EFB04FCE6FF0DFFB93C4F4FFFC
:108AD000B3F4E40023209400EFA04FB90325040071
:108AE0008320C10103248101832441010329010161
:108AF0008329C100032A8100832A41001301010256
:108B000067800000130101FF232611002324810048
:108B1000EFE08FE217E7FFFF1307C751930600004E
:108B20001306100093054006178501001305858D77
:108B3000EFC08FFF6302050213040500EFA00F8151
:108B400013060500130700009306000093051000AC
:108B500013050400EFC05F8FEF901FCB8320C1008F
:108B60000324810013050000130101016780000048
:02000004800278
:100000001C64FEFF8C65FEFF2864FEFF8C65FEFF0E
:100010008C65FEFF8C65FEFF8C65FEFF5064FEFF65
:100020008C65FEFF8C65FEFF7864FEFF8864FEFF32
:100030008C65FEFFA064FEFFB064FEFFB064FEFFAF
:10004000B064FEFFB064FEFFB064FEFFB064FEFF6C
:10005000B064FEFFB064FEFFB064FEFF8C65FEFF7F
:100060008C65FEFF8C65FEFF8C65FEFF8C65FEFFD8
:100070008C65FEFF8C65FEFF8C65FEFF8C65FEFFC8
:100080008C65FEFF8C65FEFF8C65FEFF8C65FEFFB8
:100090008C65FEFF8C65FEFF8C65FEFF8C65FEFFA8
:1000A0008C65FEFF8C65FEFF8C65FEFF8C65FEFF98
:1000B0008C65FEFF8C65FEFF8C65FEFF8C65FEFF88
:1000C0008C65FEFF8C65FEFF8C65FEFF8C65FEFF78
:1000D0008C65FEFF8C65FEFF8C65FEFF8C65FEFF68
:1000E0008C65FEFF8C65FEFF8C65FEFF8C65FEFF58
:1000F0008C65FEFF8C65FEFF8C65FEFF8C65FEFF48
:10010000F464FEFF1C65FEFF8C65FEFF8C65FEFF40
:100110008C65FEFF8C65FEFF8C65FEFF8C65FEFF27
:100120008C65FEFF7C65FEFF8C65FEFF8C65FEFF27
:100130002C62FEFF3463FEFF8C65FEFF8C65FEFFC4
:100140008463FEFF8C65FEFFFC63FEFF8C65FEFF93
:100150008C65FEFF4464FEFFE869FEFF546AFEFF03
:10016000F469FEFF546AFEFF546AFEFF546AFEFF04
:10017000546AFEFF8C68FEFF546AFEFF546AFEFF5D
:10018000B468FEFFC468FEFF546AFEFFDC68FEFF31
:10019000EC68FEFFEC68FEFFEC68FEFFEC68FEFF1B
:1001A000EC68FEFFEC68FEFFEC68FEFFEC68FEFF0B
:1001B000EC68FEFF546AFEFF546AFEFF546AFEFFBD
:1001C000546AFEFF546AFEFF546AFEFF546AFEFF43
:1001D000546AFEFF546AFEFF546AFEFF546AFEFF33
:1001E000546AFEFF546AFEFF546AFEFF546AFEFF23
:1001F000546AFEFF546AFEFF546AFEFF546AFEFF13
:10020000546AFEFF546AFEFF546AFEFF546AFEFF02
:10021000546AFEFF546AFEFF546AFEFF546AFEFFF2
:10022000546AFEFF546AFEFF546AFEFF546AFEFFE2
:10023000546AFEFF546AFEFF546AFEFF546AFEFFD2
:10024000546AFEFF546AFEFF546AFEFF546AFEFFC2
:10025000546AFEFF546AFEFF3069FEFF6C69FEFFC0
:10026000546AFEFF546AFEFF546AFEFF546AFEFFA2
:10027000546AFEFF546AFEFF546AFEFFD869FEFF0F
:10028000546AFEFF546AFEFF6066FEFFB467FEFF1D
:10029000546AFEFF546AFEFF4468FEFF546AFEFF84
:1002A0007068FEFF546AFEFF546AFEFF486AFEFF54
:1002B000000102020303030304040404040404040D
:1002C00005050505050505050505050505050505DE
:1002D00006060606060606060606060606060606BE
:1002E00006060606060606060606060606060606AE
:1002F000070707070707070707070707070707078E
:10030000070707070707070707070707070707077D
:10031000070707070707070707070707070707076D
:10032000070707070707070707070707070707075D
:10033000080808080808080808080808080808083D
:10034000080808080808080808080808080808082D
:10035000080808080808080808080808080808081D
:10036000080808080808080808080808080808080D
:1003700008080808080808080808080808080808FD
:1003800008080808080808080808080808080808ED
:1003900008080808080808080808080808080808DD
:1003A00008080808080808080808080808080808CD
:1003B000546D725100000000546D7220537663003A
:1003C000286E756C6C2900004572726F7220696E20
:1003D00020787878207461736B73200D0A00000018
:1003E0006D69616F750A00006D69616F75320A0091
:1003F00068756E6772790A0054696D657232000023
:10040000436865636B54696D657200005761697478
:100410004F0000005365744200000000526E647685
:0404200000000000D8
:100424001000000000000000017A5200017C01016C
:100434001B0D02001000000018000000A478FEFF4D
:100444005804000000000000100000002C00000010
:10045400E87CFEFF340400000000000010000000EF
:10046400400000000881FEFF1004000000000000AE
:08050C00FC8F01000900000052
:040000058000004037
:00000001FF
